:10000000C02400201935000015350000153500000A
:1000100000000000000000000000000000000000E0
:100020000000000000000000000000001535000086
:10003000000000000000000015350000153500002C
:100040001535000015350000B9140000412E0000E0
:100050001535000015350000153500001535000078
:10006000952D0000A52D0000B52D0000C52D000028
:10007000D52D0000E52D00001535000015350000D8
:100080001535000015350000153500000000000092
:100090000000000015350000153500001535000082
:1000A0001535000015350000153500001535000028
:1000B0000000000010B5064C2378002B07D1054B3B
:1000C000002B02D0044800E000BF0123237010BDC4
:1000D0002C02002000000000F8980000084B10B52A
:1000E000002B03D00749084800E000BF0748036819
:1000F000002B00D110BD064B002BFBD09847F9E731
:100100000000000030020020F8980000F89800007D
:100110000000000010B505200D4B98478023DB053B
:10012000A02292011A8104225A701A005378042BDB
:10013000FCD1BFF34F8F30BF0520064B9847064ACE
:1001400093690C218B4308390B43936110BDC04662
:100150007D300000C12F0000001400400122014B3F
:100160001A707047910200200122014B1A607047FB
:10017000FC02002010B5064C022206492000064B66
:1001800098473722A35C04210B43A35410BDC046FB
:10019000040300205D010000C9260000F0B591B005
:1001A0002A4C0523237000236370A37001A9012248
:1001B0004A708B700A700520254B98472378D9091F
:1001C0000022002904D15A09D20122498C466244F6
:1001D0001F263340012529009940916102AC25700A
:1001E00000230393049323746374A574E574237547
:1001F0002422A354183A002108A8174B9847174BFC
:10020000A36180235B02E360154BA36201235B4281
:10021000E362144B2363144B6363144F2200842165
:10022000C9053800124B98473C682000114B98478D
:100230000640B540104B1D603A68D369002BFCD1D5
:10024000236802221343236011B0F0BD4003002055
:10025000952E0000002800405B360000A0860100BB
:10026000030004000300060003000700040300204D
:100270009D230000652D000000E100E010B584B072
:1002800001AC2000074B98470E23019300236360C5
:1002900023720233E37221000E20034B984704B00F
:1002A00010BDC046791100008D11000010B500226C
:1002B0000E210448044B984700210E20034B984719
:1002C00010BDC04669010000F52D0000212E000080
:1002D00010B5164B802212025A615A615A615A6156
:1002E0009A619A619A619A61802212055A6100208E
:1002F0000F4B98470200002392185B410D480021E4
:10030000801859410C4A00230C4CA0470C4B9847CD
:100310000C4B1B78002B04D101220B4B1A600020E0
:1003200010BD0A480A4B9847F6E7C046002800402F
:10033000DD320000571B0000581B00009D670000C5
:10034000010000204C02002048020020A88E00007E
:10035000B9410000F0B583B0174B9847174B984749
:100360000125174B1D70BFF35F8F62B601AC65703E
:100370000023A3702570134F80231B05BB61210050
:100380001B20114EB047257080231B02BB6121004A
:100390000F20B0470D4B98470D4B98470D4B1B78DE
:1003A000002B04D10C4B9847002003B0F0BD0B4844
:1003B0000B4B9847F6E7C0467D020000AD020000F7
:1003C0005800002000280040952E00009D010000EC
:1003D000750100004C020020D1020000948E000044
:1003E000B9410000044B802212059A61802212025A
:1003F0005A619A610020704700280040002909D006
:100400000300411800201A78801AC0B201338B42D1
:10041000F9D170470020FCE7F0B5CE46474680B5DD
:1004200085B0019002910392444C0122444920007E
:10043000444B98470020444B984703001800002184
:100440001A000B0012184B4112184B41150F1901DD
:1004500029431001801A99413C4A002380185941D0
:100460003B4A00233B4DA8473B4B98476B469B8933
:10047000029A01992000394CA047394B1870002886
:1004800021D1384C384B99462F4B98464B461B7818
:10049000002B21D10020C047060000272B48002157
:1004A000801979412A4A00232A4DA8472A4B9847A8
:1004B000013C002CEAD1002221492048214B9847D9
:1004C0001220404221E000221D491C481D4B984744
:1004D000234B1878404218E00022234B1A70019BEE
:1004E0001B78224AD45C002C14D1002214491348F2
:1004F000144B984702990B781D4A13704978517034
:100500007F2293431B4A1370039805B00CBC90469E
:100510009946F0BD00200C4B9847020000232000B4
:100520000021154CA047094A002380185941084A68
:100530000023084CA047084B9847D6E70403002047
:1005400040030020D1250000DD320000BFCF6A004B
:10055000C0CF6A009D67000001000020E126000076
:1005600043030020B90B0000910200200C00002082
:10057000F0020020F8020020DD67000000B583B023
:1005800001A8054B1A8802809B7883700322694674
:10059000024B984703B000BD8C8E00001904000088
:1005A00000B583B001A8054B9A8802809B798370BF
:1005B00003226946024B984703B000BD8C8E0000B1
:1005C0001904000010B582B0040001A801230370D3
:1005D00000234370837003226946034B98476B46A0
:1005E0009B78237002B010BD1904000010B582B0D2
:1005F000040001A8032303700023437083700322C7
:100600006946034B98476B469B78237002B010BD38
:100610001904000000B583B0010001A80422027093
:10062000002242708270C2700432024B984703B0BD
:1006300000BDC0461904000070B58AB004000E0069
:1006400001AD232200212800064B984705232B707B
:100650006C700334E2B231002800034B98470AB0B3
:1006600070BDC0465B3600001904000070B58AB04A
:1006700004000E0001AD232200212800064B9847FC
:1006800006232B706C700334E2B231002800034B58
:1006900098470AB070BDC0465B36000019040000E0
:1006A000F0B58DB005000E001700019303AC2322B6
:1006B00000212000074B9847082323706570A6701F
:1006C000E7700535EAB201992000034B98470DB059
:1006D000F0BDC0465B3600001904000070B592B052
:1006E00005000C0009AE2322002130000D4B984775
:1006F0000B2333707570002D0CD0230026226A4422
:10070000691EC9B2013161181878107001330132C5
:100710008B42F9D10235EAB2694609A8024B9847E3
:1007200012B070BD5B3600001904000070B592B0C5
:1007300005000C0009AE2322002130000D4B984724
:100740000C2333707570002D0CD0230026226A44D0
:10075000691EC9B201316118187810700133013275
:100760008B42F9D10235EAB2694609A8024B984793
:1007700012B070BD5B3600001904000000B583B0F4
:1007800001AB0D221A70587099700A3A6946180028
:10079000014B984703B000BD1904000030B585B087
:1007A0000400134B1B78002B0FD11B211148124D55
:1007B000A847124A5378127821001148A8471B21F4
:1007C0000C480D4B984705B030BD6B460022032105
:1007D00001200C4DA8471B210B48074DA8471B21A2
:1007E0000A48A8476B465A7921000948A847E6E716
:1007F000F8020020F08E00009D400000F002002072
:10080000F88E0000A1060000C08E0000C88E000017
:10081000D08E0000F0B583B000900191A74B9847AF
:100820000020A74B9847462200230021A54EB04741
:10083000A54A002380185941A44A0023A44EB0477A
:10084000A44B9847A44B1B78002B00D098E0A348FA
:10085000A34B98470500A04B1B78002B00D0A5E0C8
:100860001B21A048A04EB0471B21A048B047A04B79
:100870001B78A04AD15C21209F4B9847964B1B7850
:10088000002B00D0A5E09D4909209D4B9847924B35
:100890001B78002B00D0B2E00020894B98476422DF
:1008A00000230021874EB047874A00238018594112
:1008B000864A0023864EB047864B98470199009898
:1008C000904B9847844B1B78002B00D09BE0002274
:1008D0008D4B1A601A001368002BFCD000228A4B43
:1008E0001A600026764F01360020B847874A002359
:1008F0000021744CA047744A002380185941734A60
:100900000023734CA047734B9847744C2000744BE2
:1009100098476378DB0601D4282EE4D16E4B1B7810
:10092000002B00D08DE00020654B98474622002325
:100930000021644CA047644A002380185941634A4F
:100940000023634CA047634B98475C4B9847624B2E
:100950001B78002B00D09AE00020594B9847462284
:1009600000230021574CA047574A002380185941C3
:10097000564A0023564CA047564B984703B0F0BD4B
:100980006348644B984700204D4B984764220023EE
:1009900000214C4EB047604A0023801859415F4AFD
:1009A00000234B4EB0474B4B984750E75C484E4BAB
:1009B0009847002D09D0494E75195A4F4A4C317845
:1009C0003800A0470136AE42F9D15748574B9847F7
:1009D00046E757484F4B98470020394B98476422C9
:1009E00000230021374EB0474B4A0023801859415D
:1009F0004A4A0023364EB047364B984743E74D48A6
:100A0000444B984748E74C48424B984700202C4BB2
:100A100098476422002300212A4CA0473E4A002325
:100A2000801859413D4A0023294CA047294B98473B
:100A3000294B1B78002B00D149E740483B4B984796
:100A400045E77200921931003D48274CA047284BDA
:100A50001B78284AD35C9A06920F0721194039481F
:100A6000A0471E481E4B984705002D48A047002D63
:100A700009D01A4C65192B4E1B4F21783000B8470E
:100A80000134AC42F9D12848284B98474BE720481D
:100A9000204B984700200A4B9847642200230021EE
:100AA000084CA0471C4A0023801859411B4A0023C8
:100AB000074CA047074B98474EE7C046A1050000EA
:100AC000DD320000DD670000BFCF6A00C0CF6A00E2
:100AD0009D670000010000204C0200205002002011
:100AE00015060000C88E00009D400000F08E00003A
:100AF00090020020380000207D0700002C0000201C
:100B00002D070000DD060000FC020020B80B0000ED
:100B10003C8F00009D070000571B0000581B000081
:100B2000508F0000688F0000A0910000B9410000C4
:100B3000708F00008C8F0000A48F0000B88F000021
:100B4000C88F0000F08F0000F0B5D6464F464646ED
:100B5000C0B582B00500894690469A46504B1900B0
:100B6000403100221A7001338B42FBD14D4F4E4E63
:100B70000020B847FA22520000230021B0474B4A18
:100B80000023801859414A4A00234A4CA0474A4B47
:100B90009847434C2000494B98476378DB06E7D5DC
:100BA0003F4FFE7800203F4B9847454A00230021E5
:100BB0003D4CA0473D4A0023801859413C4A002340
:100BC0003C4CA0473C4B984738003E4B98473C78FC
:100BD000200002230193002C27D10A9B1860304C7F
:100BE0002000394B984724782C80651E1F2D2FD963
:100BF000364B1B78002B3DD1354B9847334B1B7838
:100C0000002B48D1072333404246137003231E4074
:100C100053461E70224B03334A461360019802B0BC
:100C20001CBC90469946A246F0BD1D4F3900294B89
:100C30009847FB1CE11C791800201A7880180133B2
:100C40008B42FAD12100244B984700230193C4E73B
:100C5000134F39002000214B9847F81C2900204BE6
:100C600098473B199B788342C2D00123019A1A43CB
:100C70000192BDE71B481C4B9847094DEC1C2335DE
:100C80001A4F21781A48B8470134A542F9D11948BA
:100C9000154B9847B0E71848184B9847B2E7C0463D
:100CA00050020020DD320000DD670000BFCF6A0087
:100CB000C0CF6A009D6700000100002015060000FB
:100CC00088130000ED050000C50500004C0200205F
:100CD000A105000039060000356400006D06000023
:100CE000FD030000108F0000B94100009D4000008E
:100CF000308F0000A09100003C8F00009D07000095
:100D0000704710B500230022037043708370C370D6
:100D1000002103830362C36101240471C0246401C0
:100D2000C480017242728272C27202732A24025516
:100D300042738273C27303610275063C0255C38419
:100D40000385417510BD0000F0B5CE4600B59AB0E0
:100D5000050016000160B54A136A082003431362B8
:100D60000B780338DB0703D51AB004BC9146F0BDFD
:100D70002A68138C9BB2002BFBD10B781C209B079D
:100D8000F2D473782B71002B04D1A94AD3690421C2
:100D90000B43D3612F6833786A46137069461E206F
:100DA000A44B98471E20A44B984734796022A3494E
:100DB00002A8A34B9847132C0BD9F48860229F49B3
:100DC00002A89F4B9847132C11D900249C4B99469D
:100DD0001EE0A40002ABE05801A900234B70CB70C9
:100DE0008B7001330B70C0B2964B9847E5E7A400B7
:100DF00002ABE05801A900234B70CB708B7001331C
:100E00000B70C0B28F4B9847DFE70134142C18D019
:100E10000123A34032691A42F7D06022874902A811
:100E2000C847132CF1D8A30002AA985801A900239F
:100E30004B70CB708B7001330B70C0B2814B9847F5
:100E4000E3E7737B9B01B27BD2011343DBB23B70C0
:100E5000337DDB0172781343DBB2BB70F378342B44
:100E600000D933E19B00784AD3589F4604221024CE
:100E700002211AE0717A327A102416E00622102438
:100E8000012112E00822102400210EE0002230246B
:100E900000210AE000222024002106E00022002494
:100EA000002102E0022210240121090170230B40DD
:100EB00013433B732A68138C9BB2002BFBD1737DC9
:100EC00017203F2B00D94FE7F27BD2011343DBB24F
:100ED0007B732A68138C9BB2002BFBD1B3787B7099
:100EE0002423F35CDB00327B92001A43F37A134332
:100EF000B27A5200134323437B812A68138C9BB23E
:100F0000002BFBD1338B002B1FD0102C00D1BFE066
:100F10006BD9202C00D19DE0302C16D1F27A002A1A
:100F20000AD0F26980321720FF2A00D91CE7326A02
:100F30008032FF2A00D917E71720F269FF2A00DD67
:100F400012E7326AFF2A00DD0EE77A8913437B81BC
:100F50002A68138C9BB2002BFBD1B38BFB812A68D0
:100F6000138C9BB2002BFBD1338C3B822A68138CF1
:100F70009BB2002BFBD13379F28813433B812A6863
:100F8000138C9BB2002BFBD12A33F35CFB7007233D
:100F90003B711D33F35C002B1BD0F38C2B4A1720C5
:100FA000934200D9E0E67B822A68138C9BB2002B27
:100FB000FBD1328D80231B01D31824499BB217200B
:100FC0008B4200D9D0E6BA822A68138C9BB2002BE0
:100FD000FBD11F4B1B681A02E021C9000A409B0687
:100FE0005B0F1343BB850020BEE6002CADD1F27A27
:100FF000002A0FD0F269802109018C46624413490E
:1010000017208A4200D9AFE6326A62440F498A4209
:1010100000D9A9E60D4A1720F169914200DDA3E647
:10102000316A914200DD9FE68FE7C0460004004030
:1010300000140040B933000049330000EC90000078
:1010400049360000B534000018900000FF0F000082
:1010500020608000F27A002A0FD0F2698021890096
:101060008C4662441A4917208A4200D97CE6326ACB
:10107000624417498A4200D976E6154A1720F16979
:10108000914200DD70E6316A914200DD6CE65CE77A
:10109000F27A002A0FD0F269802109028C4662445C
:1010A0000C4917208A4200D95EE6326A6244094937
:1010B0008A4200D958E6074A1720F169914200DDBB
:1010C00052E6316A914200DD4EE63EE717204BE6DC
:1010D000FF030000FFFF0000064A137802210B43C4
:1010E0001370012053681942FCD153681842F9D19A
:1010F0007047C04600240040064A137802218B4303
:101100001370012053681942FCD153681842F9D179
:101110007047C0460024004010B5124A5169802330
:101120009B000B435361104A137801210B4313704A
:101130000131012053681942FCD153681842F9D19A
:10114000094A137810210B431370084B19004031E2
:10115000002204C38B42FCD10822054B1A60054BC8
:10116000984710BD000400400024004044030020C4
:1011700000E100E0D9100000002303604360012279
:10118000027283720132C27243727047F0B583B04B
:1011900005000C001C4B984701A900234B70CB7035
:1011A00023790B70237A8B702078184B9847002195
:1011B0001F2D00D8164907222A409200E77AA37A09
:1011C000002B01D008231F43EB089B00CB18D869E4
:1011D0000F269640B04397403A000243DA61637AA3
:1011E000002B0BD18A690123AB40DB431B041B0C92
:1011F00013408B61074B984703B0F0BD8A69012308
:10120000AB4013438B61F5E7F9100000B5340000E3
:1012100000240040D910000003681869431E98415B
:10122000C0B2704770B5040006680422084B1A600B
:10123000084D2000A8470028FBD133880222134321
:101240003380044D2000A8470028FBD170BDC04664
:1012500000E100E01912000070B5040006680421E6
:101260008023084AD150084D2000A8470028FBD110
:101270003388022293433380034D2000A84700287F
:10128000FBD170BD00E100E01912000070B5040050
:1012900006680A4B98470023A386E386084D200082
:1012A000A8470028FBD13388012213433380044D23
:1012B0002000A8470028FBD170BDC046591200008D
:1012C00019120000F8B504000E0007680C4D20004C
:1012D000A8470028FBD12379002B09D01720012B28
:1012E00005D1BE61064D2000A8470028FBD1F8BDFE
:1012F000044B17209E42FAD8B6B23E83F2E7C046AE
:1013000019120000FFFF0000F0B583B00400019146
:1013100015000668134F2000B8470028FBD1237939
:10132000002B0ED0012B19D11730012D17D80835FD
:10133000AD00019BAB510B4D2000A8470028FBD10D
:101340000DE01720022D0AD8074B019A9A4206D8C1
:101350006B469B8810356D00AB53ECE71A2003B049
:10136000F0BDC04619120000FFFF000070B5040078
:10137000150001601F4A516980235B000B435361D4
:1013800000221D4B1A611D4B9847AB7823711C4BF3
:101390001C6022682B79DB0329880B439BB21380E6
:1013A000AB78002B13D01720012B0FD113889BB2E1
:1013B0001380EB78002B03D0138880210B4313801C
:1013C000A968002220000F4B9847002070BD1388A9
:1013D00004210B431380EB781720002BF6D1002259
:1013E000A9682000074EB047E96801222000B047F5
:1013F0000020EBE700040040001000408D120000C8
:101400008403002009130000F8B504000E000379DE
:101410001520002B00D0F8BD2768064D2000A847F6
:101420000028FBD1BE83034D2000A8470028FBD134
:10143000F1E7C046191200000A2A09D0072A07D985
:101440000379002B10D0012B12D11633092A09D8A9
:10145000931C9B001950838E012191400B439BB23A
:10146000838600231800704717230A2AFAD8EFE76B
:101470001723F7E710B502680A2911D0072912D9F6
:1014800080235B000C00083CA340C024A400234040
:101490005381C38E01228A4013439BB2C38610BD81
:1014A000044B5381F5E701248C40FF2323405381F3
:1014B000EFE7C0460080FFFFF8B5DE4657464E46D0
:1014C0004546E0B52B4B1B689A461E68DB8E52469C
:1014D000928E1A409046B289738913401AB2002A3C
:1014E00008DBFF271F402AD0002401239946FE3342
:1014F0009B4614E043465B0507D41F4BB3813CBCBD
:1015000090469946A246AB46F8BD53461B6B98479A
:10151000F3E75B461D40B5810134082CEFD0230072
:101520004D46A5402F42F4D0424622414946114241
:10153000EFD002339B0052469B589847E9E7DA0503
:101540000AD54346DB0503D480235B00B381D6E78D
:1015500053469B6A9847F7E79B05D0D543469B05C2
:1015600003D480239B00B381C9E75346DB6A9847C5
:10157000F7E7C046840300200080FFFFF0B5C646B1
:1015800000B50C00904600280FD1002A11DD8F18FD
:10159000094E0A4D306821002B6898470134BC423F
:1015A000F8D1404604BC9046F0BD01235B4298460A
:1015B000F7E78046F5E7C046900300208803002047
:1015C000F0B5C64600B50E0015000138022810D847
:1015D000002A11D000240C4B98460C4F4346186843
:1015E000315D3B689847002808DB0134A542F5D1FE
:1015F00006E00124644203E0140001E00124644297
:10160000200004BC9046F0BD900300208C03002015
:101610000122014B1A6070475404002070B582B05B
:1016200005000E0000226B46DA80064C6B46991DC1
:101630002800A0470028F9D16B4606331B88337079
:1016400002B070BD2B23000070B505008CB2034EB4
:1016500021002800B0470028FAD170BD0123000006
:1016600030B58DB001AC20000D4B98470523637059
:101670000C4D22000C4928000C4B98472A68138C0B
:101680009BB2002BFBD1137802210B431370054B47
:101690001A68138C9BB2002BFBD10DB030BDC04635
:1016A000030D000094040020000C0043490D0000CD
:1016B000F0B587B005220F2302A98C4663441A7047
:1016C00001320E2363441A70544B9847544C002146
:1016D0002000544B9847544B19882000534B98478F
:1016E000534A54491368002B02D10B68002BF9D0E0
:1016F000504B1B68002B1CD000224E4B1A604E4BE7
:101700001B68002B11D1464C00212000454B984707
:101710004A4B19882000454B98470022444B1A60D9
:10172000474B9847012007B0F0BD4648464B9847C5
:10173000E9E7414B1B68002B53D10E2702AB9C46B7
:1017400067440F26664405AD404B00933B003200D2
:1017500004A928003E4CA04703903B7832782988A2
:101760003C483D4DA847344B1B68002B3DD10498A5
:1017700000233A49C25CCA5401331C2BFAD1374EBC
:10178000B368726831683648334DA84731693548C7
:10179000A847354FB069B84702000B003348A84747
:1017A0002A4B1868324B9847FC218905314B9847E2
:1017B0003149324B9847B84702000B003048A847E0
:1017C00071693048A847039C21002F48A8472F483B
:1017D0001D4DA8472E48A8470022164B1A6020002E
:1017E000A1E72C48184B9847A7E705AD29882A4858
:1017F000194B98472B88002B0BD00025274F164CF0
:1018000005AE049B595D3800A04701353388AB42D3
:10181000F7D823480C4B9847A9E7C0467D05000040
:101820009C030020C5120000500000200914000095
:10183000FC02002054040020280400205400002052
:10184000A105000054910000B9410000500400209F
:10185000490B0000A49100009D400000700400208E
:10186000F891000010920000958D00002C9200006D
:10187000B9710000416C000000000643816E000059
:101880005092000064920000849200007891000061
:101890009492000074910000D4910000F091000037
:1018A000A0910000F8B5214C21001C31230000223A
:1018B0001A7001338B42FBD11D4A1E4B1A601E4A1F
:1018C0001E4B1A601E4A1F4B1A60184D1E4B1A6899
:1018D0002A605A686A609A68AA60DB68EB601B4BF2
:1018E0001B886B611A4A1368591C11602B61194BD4
:1018F0001868194B9847FC218905184B98471849D7
:10190000184B9847A8611C212800174B9847287747
:101910001D35164E164F21783000B8470134AC42C1
:10192000F9D11448144B98471D20F8BD70040020CD
:1019300033331340940300200000E143D40300201C
:101940006666D6408C0400203C0400202C04002055
:101950009402002050040020B9710000416C000086
:1019600000000643816E0000FD0300004C91000062
:101970009D400000A0910000B9410000F0B583B087
:101980002D4B98472D4B186000281AD02C4B1B6804
:10199000002B19D12A4B1B68002B19D1294C274B3E
:1019A0001878012301933B33009300230022210088
:1019B000254DA84723001C3400221A700133A3428E
:1019C000FBD1012003B0F0BD2048214B9847E1E74F
:1019D0001A4C21681F48204DA8471A4B19691F4807
:1019E000A8472368002B0BD00024164F1C4D1A4E1D
:1019F000395D2800B0470134104B1B68A342F7D86B
:101A00001848134B98470D4B1B68002B10D000242F
:101A10000C4F154E094D04E0B04701342B68A3422A
:101A200006D9385D0300213B5D2BF5D92E20F3E765
:101A30000C48074B9847B1E7A51800003004002078
:101A4000280400207004002015080000989200006F
:101A5000B9410000C49200009D400000D8920000EF
:101A6000F0910000A0910000D140000010B584B0BA
:101A700000236A46D3700293039380225200694682
:101A80000A806A468B70054C05492000054B984733
:101A90002000054B984704B010BDC0469C030020B1
:101AA000002000406D1300002512000010B5074C07
:101AB0000A2207492000074B98470A212000064BBD
:101AC00098470022054B1A6010BDC0469C030020B9
:101AD0001116000039140000751400005404002091
:101AE000F0B5C64600B582B001AC01266670002391
:101AF0009846A3702670224F80235B047B612100EF
:101B00001820204DA847267080239B047B6121006C
:101B10001920A847267004237B6121000220A847D2
:101B2000267080231B01BB6121000B20A847434680
:101B30002370667021000820A84721000920A847CB
:101B400021000A20A84721001020A84721001120C9
:101B5000A84721001220A84721001320A847434688
:101B60002370637021000320A847267080231B0682
:101B70007B6121001F20A84702B004BC9046F0BD45
:101B800000280040952E0000F0B5DE4657464E4630
:101B90004546E0B59DB00126CC4B1E6000240025D3
:101BA000CB4B1C70CB4B9847CB4B9847CB4A136918
:101BB00002218B43136193690A318B4308390B432C
:101BC0009361C74B98470CAB8022D2050C925C60A6
:101BD000FF221A819C72DC72DB3A9E5401329E54C1
:101BE00001329C5401329C549C6205329C54013257
:101BF0009C545C611C820022DA761D761D775D762E
:101C000013229A765D77E12252021A6280225203F1
:101C1000DA60B44A1A63B44A5A63012252429A63A0
:101C2000DA63B24DB24C0CAAB2492800A047002892
:101C3000F9D1AE4CB04B1C60B04AB14B1A60B14AFE
:101C4000B14B1A600CAAAB492000A94B9847AF4E84
:101C5000336898680021AE4DA84733685868002162
:101C6000A8472368DA69002AFCD11A6802210A43CE
:101C70001A60A84B9847A84B9847A84B9847A84B81
:101C80001988A848A84B9847A84AA949A948AA4C26
:101C9000A0471C21A948A047A94B19001C310022CC
:101CA0001A7001338B42FBD14023013B002BFCD146
:101CB0004022A44B1A60A44B1B681968A34C2160F6
:101CC000A34B1868021D1A6002686260050008359F
:101CD0001D604368A3608068E0607C4C2468002C31
:101CE00003D000909B48944CA0479B4B9847002002
:101CF0009A4B9847020000239948002180185941C7
:101D0000984A0023984CA047984B98476F4B1B6804
:101D1000002B02D09648974B9847974B9847002343
:101D20009A46042402257AE008420AD19379DBB26C
:101D3000010019401C4200D029431D42F4D0214328
:101D4000F2E7908C80B28D4B1880012393719179CA
:101D5000C9B20B400C4200D02B430D4200D02343AC
:101D60001C4200D09571864B9B4698478549864B0F
:101D70009847864B99461860854EB04702000B0085
:101D80008449884684494046844FB8474346524672
:101D90009A737A4B1F88824B1868D847FC218905B3
:101DA000804B98478049814B9847B04704900591F4
:101DB000434602934B461868B047009001913A00A1
:101DC00039007B485C4B984780221206794B5A6158
:101DD0005046624B9847089000230993089A099B44
:101DE000910F079191000691069807998018594123
:101DF000001849415A4A002380185941594A002382
:101E0000594EB047594B98476B4B98476B48594BC5
:101E100098476B4B9847002838D0574B9847404E0F
:101E2000454F31686748B847674B9847674B1B6811
:101E3000002BF6D0654B52461A60654B98475D4EB5
:101E400080231B06B3615046444B98470A900023F9
:101E50000B930A980B99424A002380185941414A32
:101E60000023414FB847414B9847336A594B1A6892
:101E7000138C9BB2002BFBD1137E02210B431376F4
:101E8000138C9BB2002BFBD101204FE72C4B5B69DD
:101E9000514A934214D80132294B5A61284F79692B
:101EA0004E48254B98471F4E514630004C4B9847A3
:101EB00079691B4B196089B230001B4B9847ACE71E
:101EC000484A9342EAD91E4B5A61E7E728040020AA
:101ED0004C020020E9340000010D00000014004015
:101EE000E11A00000300160003001700980200200A
:101EF000E91F000000040043900300204916000081
:101F00008C0300201D160000880300205C000020C8
:101F1000F1410000611600006D1A0000AD1A0000CA
:101F2000540000209C03002009140000EC920000E3
:101F3000F8920000049300009D4000003C930000D4
:101F4000700400204C040020480000203C040020C5
:101F50004C0000206093000055030000DD320000BB
:101F6000571B0000581B00009D6700000100002067
:101F700084930000B9410000E50300002C04002018
:101F8000B971000000003B44B1690000A4020020C8
:101F9000958D00005C040020CC9300005D430000A0
:101FA00050040020416C000000000643816E0000D8
:101FB000D4930000002800407D19000030940000F8
:101FC000B116000090930000150100005404002099
:101FD000D102000094040020CF070000B09300005D
:101FE000C5120000204E0000F0B5DE4657464E46B2
:101FF0004546E0B591B006000C00150031600800C0
:10200000B44B9847020005280DD007001237030093
:1020100021680520C90709D511B03CBC90469946F6
:10202000A246AB46F0BD18270123F1E7216817301F
:102030008907F1D4052A47D0A749C86901229A40E7
:1020400013000343CB610FA92D239846EB5C0B7063
:10205000FFB23800A14B98473800A14B9847434640
:10206000E85C00219F4B9847EB7A73712423EB5C6B
:10207000B3712523EB5CF371EB7E33722B7F7372AC
:10208000336899461800934B9847123000220E236C
:1020900006A98C4663441A802A8A02928023DB01B7
:1020A0009A4200D1A8E017D9C023DB01029A9A42D4
:1020B00000D19CE080231B029A4200D005E103235B
:1020C00006930023079310E08349086A043A9A4074
:1020D000130003430B62B6E780239B019A4200D0B2
:1020E000F3E0102306930F3B07932B680593EB68EF
:1020F0009B466B6904932B7E03932623EB5C9846E7
:102100006B689A46002B00D19EE080235B059A45C0
:1021100004D12723EB5C002B00D183E06B7E002BE6
:1021200002D0AB7E4A4693733268029FD369002B7C
:10213000FCD10E3306AA944663441B884A46938119
:10214000059A5B461A43049B1A4353461A433A4383
:10215000039B1F023A4343465B071A432723EB5C6A
:10216000002B01D104331A436B7E9B02297F490265
:102170000B43697F09020B432421695C49040B432B
:102180002521695C09040B43E87A18432B89FF2B4E
:102190007ED0802149040A4318432C23EB5C002B9A
:1021A00003D1514B9B789B0701D580231A4331689B
:1021B000CB69002BFCD14B4658603168CB69002BB2
:1021C000FCD14B461A600EAB80221A7000225A7066
:1021D000DA709A702B6B0A936B6B0B93AB6B0C934F
:1021E000EB6B02930D9300270AAD404E5EE008238F
:1021F0000693073B079378E72B680593EB689B46AC
:102200006B6904932B7E03932623EB5C98466B68E3
:102210009A46002B14D080235B059A4500D178E7BD
:10222000002020E02B6A1F00C0B2314B984701000C
:102230000E2206AB9C46624438002E4B984712E0B3
:1022400008230693002307932723EB5C002B0ED073
:10225000069B0093079B0E2206A98C466244A96A3E
:10226000286A254FB847002800D0D5E656E72B6AE4
:102270001F00C0B21E4B98470100069B0093079BAE
:102280000E2206A88446624438001B4FB847EAE78E
:10229000EB7E002B81D08023DB041A437DE72000F6
:1022A000164B984707E00137042F0CD0F9B2BB005A
:1022B00058590028F3D0431CF5D00EA90870000C23
:1022C000C0B2B047EFE70020A6E610230693002334
:1022D00007930AE7ED2C000000040040B93300002A
:1022E00049330000452B000000200041B5340000B8
:1022F000DD3300004D29000075290000912B0000FE
:10230000C3791C22002B01D1100070470368187E8E
:10231000173AC007F8D5DA69002AFCD119850221DD
:102320001A7E0A42FCD00022EEE782791C23002AA2
:1023300001D1180070470268107E173B4007F8D59E
:10234000D369002BFCD1538BDBB2980621D09807C0
:1023500003D5022353831833EBE7580703D504232F
:1023600053831A33E5E7D80703D501235383123388
:10237000DFE7D80605D5538B10210B435383422347
:10238000D7E79B0605D5538B20210B43538341236D
:10239000CFE7138D0B800023CBE70000F0B5C646D6
:1023A00000B588B005000C00160029600B681C20E1
:1023B0009B0703D508B004BC9046F0BD0B681738E6
:1023C000DB07F7D40800754B9847052800D1DDE0FE
:1023D00007001237724AD169012383400B43D3614E
:1023E00007A924239846F35C0B70FFB238006D4BAD
:1023F000984738006C4B98474346F05C00216B4B84
:1024000098473378012B3FD03378002B03D12368D2
:102410000822134323602B000C33290028310022AB
:1024200004C39942FCD10023EB62AB620024AB866B
:102430002B863633EC540133EC540133EC54353BEA
:102440006B722C712868554B984707005849594BB7
:102450009847BF00584BFD502F6802AB80221A707E
:102460005C707F3A9A70DC703378002B02D10022C6
:1024700002AB9A70B36A0393F36A0493336B0593C8
:10248000736B069300240BE023680C221343236034
:10249000BAE73800494B98470AE00134042C10D0C1
:1024A000E1B2A3006A460C201218D0580028F0D0E0
:1024B000431CF2D002A90870000CC0B2404B9847F0
:1024C000EBE733786B71337CAB71B37CEB71337DAD
:1024D0002B7200226B46DA803378012B12D03378CE
:1024E000002B26D1B069B28B7B6AF17F0904B47FDF
:1024F0002143194379622023F35C002B1BD0402336
:102500001A4318E02868254B98471230C0B22D4B6B
:10251000984701006B469A1DB0692B4B9847030002
:102520001720002B00D045E76B4606331B783B7322
:10253000D5E7002200207368B1680B43F1680B43B4
:102540000343317C0A43717C002903D11F498978F8
:10255000890701D580210B43B17C002902D080215D
:1025600089020A43F17C002902D0802189000A43B4
:10257000317D002902D0802189010A4339680B434B
:102580003B607B681A437A60002013E7044A136AB1
:1025900002210B431362182722E7C046ED2C0000EE
:1025A00000040040B933000049330000452B00000F
:1025B00025270000292D0000A0040020912B0000F9
:1025C000B5340000DD3300004D290000002000413B
:1025D00010B544791523012C01D0180010BD047AE0
:1025E0000023002CF9D1002A5AD04B78002B46D07A
:1025F00003681B7EDB0710D40A78D1090023002969
:1026000004D15309DB012F498C4663441F2111403B
:1026100001228A409A610523DFE70A78D409002362
:10262000002C04D15309DB01264CA44663441F242B
:1026300014400122A2405A6103681A7ED20701D5D4
:102640008A789A62C2790023002AC6D102680421DE
:10265000137E0B42FCD0117E00234907BDD5538B5E
:102660005B0703D5538B04210B4353838379012BE1
:1026700002D0936A0023B0E7936A0023ADE70A789B
:10268000D1090023002904D15309DB010D498C46EF
:1026900063441F21114001228A405A6100239CE7B4
:1026A0000A78D1090023002904D15309DB01054927
:1026B0008C4663441F21114001228A409A61002305
:1026C0008BE7C04600280040931C9B00C31859604C
:1026D0003621012393401A00435C1343435470474F
:1026E00030B51724002B01D1200030BDC579053449
:1026F000002DF9D01C34055D333C052DF4D08386C4
:1027000003868262C16205223823C254363B43727B
:1027100003689A7542790024002AE5D102321A76BC
:102720009A75E1E7F8B58000864BC45826683723D0
:10273000E35C3622A75C1F40337EB57D1D40EB076E
:102740002ED56379012B25D0002B29D1637A002B5C
:1027500026D02168E26A1378DBB2501CE062A079CF
:10276000012800D16BE09BB2DB05DB0D8B62A38EF1
:10277000013B9BB2A386A38E9BB2002B10D10133E9
:102780003375637A012B0BD1E379002B08D1023327
:10279000B37505E0637A002B40D0637A002BD8D163
:1027A0006B0713D5738B5B0753D5637A012B08D066
:1027B0001E223823E254353B6372023333753B07E4
:1027C00043D4B36A738B042213437383AB0715D5C9
:1027D0006379002B0ED107333375053B3376013314
:1027E00063720023A386238638330022E254FB065B
:1027F00000D57FE06379012B00D17FE02B0708D55E
:102800006379002B05D1083333753376BB0600D5C9
:102810008AE06DB2002D00DA8AE0F8BD4A4B1B88D1
:10282000B362638E013B9BB26386638E9BB2002BC7
:1028300001D1013333756379012BAED084E7507831
:10284000000203430232E2628EE72000A369984748
:10285000B7E7637A012B27D023689B6ADB05DB0D82
:10286000DAB2A16A0A70A26A511CA162A179012997
:1028700033D0238E013B9BB22386238E9BB2002B49
:10288000A4D100223833E254343B3375637A022BEF
:1028900029D0637A002B00D098E7BB0700D495E7D6
:1028A00020002369984791E723689B6A638E013B68
:1028B0009BB26386638E9BB2002B00D086E7043305
:1028C000337500223433E254353B6372FB0700D486
:1028D0007CE72000E368984778E71B0A5370A36AF7
:1028E0000133A362C5E77B0700D46FE7200063696B
:1028F00098476BE72000E36998477BE7637A012BF1
:1029000000D086E7E379002B00D082E702333375ED
:102910000133637200223533E254FB0700D46DE7C4
:102920002000E368984769E72000236A984770E72A
:102930008023337533767B0600D46EE7636A20000C
:1029400098476AE7A00400209C04002010B54908BD
:1029500040230024814202D2180010BD1C00091A35
:10296000631C9BB28842F9D94023FF2CF4D8148011
:102970000023F1E7F0B5DE4657464E464546E0B542
:1029800089B00C00059212AA117805004D4340222F
:10299000A54207D9100009B03CBC90469946A24612
:1029A000AB46F0BD002B55D1020008000021634D5D
:1029B000A8478346260000270023002400930194A3
:1029C000002200233F2020218C461F3902960397C6
:1029D00014E06446241A0D00E540A84615E0029C68
:1029E000039D121BAB414D46009E019F35433C00A9
:1029F000464634430095019401381DD32024644297
:102A00000419E6D40D00A540A8460C008440A14658
:102A100092185B4114001D0046465F463E4203D0BB
:102A20000E00264332002B00029C039D9D42E3D8FA
:102A3000D5D19442E0D8D2E7002201230098019931
:102A4000121A8B411900130C0A041A43059B1A80B1
:102A500000229FE70022012BF8D1630F0493E300CB
:102A600098460A0000230021344CA04704000D00C2
:102A700000239C46069320339B460126634607931A
:102A800048E05946C91B3000C840824610E0009813
:102A90000199121A8B410299484601430291013F64
:102AA00025D3202149427918EBD430008840824652
:102AB0003100B940894692185B4110001900444624
:102AC0004D462C40A4465446049D2C40A2466446E4
:102AD00055462C4303D03400044322000B000098D9
:102AE00001999942DBD8D2D19042D8D8CFE7009C47
:102AF000019D0299079A8B1ADB0811498B4214D960
:102B0000069B0133DBB219000693130001330793D0
:102B1000082908D000230293002200233F210094BB
:102B200001950F00BDE7402234E7402206990829AD
:102B300000D12FE74A031A4388E7C046DD6700004B
:102B4000FF1F000010B582B004000E4B1B78002B55
:102B500007D0002905D10B4B5B78834210D01D2094
:102B60000CE001A90C701120074B98471120074B6E
:102B70009847044B5C7001221A70002002B010BD0F
:102B80000020FBE7A8020020B93300004933000011
:102B90003C4B984232D00AD93B4B98424ED03B4BEB
:102BA000984255D03A4B984238D000207047842341
:102BB000DB0598420CD0374B9842F6D1012917D04B
:102BC000002957D0022915D0032915D00020EDE7A0
:102BD000012907D000294BD0022905D0032905D0AF
:102BE0000020E3E72C48E1E72C48DFE72C48DDE74D
:102BF0002C48DBE72C48D9E72C48D7E7012907D038
:102C0000002939D0022905D0032905D00020CDE7BD
:102C10002748CBE72748C9E72748C7E7012907D056
:102C200000292BD0022905D0032905D00020BDE7BB
:102C30002248BBE72248B9E72248B7E7022903D078
:102C4000032903D00020B1E71F48AFE71F48ADE7D5
:102C5000012907D0002913D0022905D0032905D066
:102C60000020A3E71A48A1E71A489FE71A489DE702
:102C70001A489BE7032099E7194897E7194895E711
:102C8000194893E700080042001000420004004386
:102C9000000C00420004004203000500030006008F
:102CA000030007000300010003001E0003001F00D3
:102CB0000300090003000A0003000B0003001100D9
:102CC000030012000300130003000E0003000F00B6
:102CD000030017000300180003001900030004009C
:102CE00003000800030010000300160030B587B091
:102CF0000B4B6A4632CB32C232CB32C2009B83428C
:102D00000BD001239A0069465258824206D0013303
:102D1000062BF7D1002007B030BD0023D8B2FAE768
:102D20004894000070470000F0B50A4B1B78002B58
:102D30000CD1094F094E0A4D0024DE515A19146076
:102D40000433182BF9D10122024B1A708000024B78
:102D5000C150F0BDAA020020AC020020252D0000C9
:102D6000A004002000B583B008236A461370013325
:102D70005370013393700133D370013313710133F6
:102D80005371034B98476B46185603B000BDC046BD
:102D9000ED2C000010B5024B1B680020984710BDB9
:102DA000AC02002010B5024B5B680120984710BDB3
:102DB000AC02002010B5024B9B680220984710BD62
:102DC000AC02002010B5024BDB680320984710BD11
:102DD000AC02002010B5024B1B690420984710BDBF
:102DE000AC02002010B5024B5B690520984710BD6E
:102DF000AC0200201723002A01D0180070478B0076
:102E0000064A9B58002B03D0834205D01D23F4E7CC
:102E1000890088500023F0E70023EEE744030020F8
:102E20001723002901D01800704700221F2800D85E
:102E3000024A0123834013610023F4E70024004089
:102E400070B50022104B1A70002310491F25104E38
:102E50000D4C0AE00D4908E023780133DBB2237002
:102E60000F2B10D800211F2BF4D928001840012265
:102E7000824048691042EFD04A619B009B59002B69
:102E8000EAD09847E8E770BDB8040020002400406D
:102E90004403002000B583B001AB80221A700A7889
:102EA0005A704A789A708A78DA701900014B9847FC
:102EB00003B000BDB5340000704700000C4B1B6828
:102EC000002B06D1EFF31083002B07D00022094B13
:102ED0001A70074A136801331360704772B6BFF364
:102EE0005F8F0022044B1A700132024B1A70F0E718
:102EF000C4020020C802002058000020084B1A68B5
:102F0000013A1A601B68002B09D1064B1B78002B75
:102F100005D00122044B1A70BFF35F8F62B6704771
:102F2000C4020020C80200205800002010B5082864
:102F300003D880001C4B1B589F46002032E01B4BDF
:102F400018692FE01A4B187D0007800F431C1948A1
:102F5000584327E0154B586924E0144B1B680020A8
:102F60009B071FD5124980225200CB681342FCD028
:102F70000E4B1B685B0701D40F4813E000200F4B7A
:102F800098470A4B9B681B041B0C58430AE02823F4
:102F9000074AD35C00209B0704D5044BD86801E0A6
:102FA0008020000210BDC04660940000CC020020CA
:102FB000000C004000093D00006CDC02DD33000025
:102FC000082803D88000294B1B589F4617204BE048
:102FD000274A137D02210B431375002044E0254A44
:102FE000936902210B43936100203DE0204A138A3C
:102FF00002210B431382002036E01E4A536902214E
:103000000B43536100202FE01B490B68022213433E
:103010000B60174B1A831900FE32CB681342FCD0A9
:10302000154A9168124B19625268DA6100221A83BC
:1030300019000132FF32CB681342FCD00E4B1B68E3
:103040009BB20B4A138300200EE0094928228B5CB7
:10305000022003438B5408003821263A435C134274
:10306000FCD1002000E000207047C046849400009E
:10307000000C004000100040CC020020082832D88C
:1030800080001A4B1B589F46194A137D02218B431F
:10309000137500207047174A936902218B4393618F
:1030A0000020F7E7124A138A02218B431382002083
:1030B000F0E7104A536902218B4353610020E9E78E
:1030C0000D4B1A6802218A431A601B689BB2084A9A
:1030D00013830020DEE7064928228B5C022083430D
:1030E0008B540020D6E71720D4E7C046A8940000F0
:1030F000000C004000100040CC02002010B584B04D
:1031000080225200284B9A60FD3A284B9A60284A48
:1031100053681E218B4353608023DB059B78022B71
:1031200009D08023DB0501229A7101329A701A00BE
:103130009379002BFCD01C4B197D802252420A430C
:103140001A751A7D40218A431A751A4B98471A4CF2
:103150000123A3716371237101A94B6000234B709C
:1031600006220A700B724B720020144B9847002005
:10317000134B98470020134B98472379013BD840C5
:10318000114B98420ED88023DB059B78002B09D089
:103190008023DB0501229A7100229A701A0093792C
:1031A000002BFCD004B010BD000C00400014004007
:1031B00000400041CD31000000040040F13100002A
:1031C0009D320000DD320000001BB700064A536943
:1031D00040210B4353610122044B1A7019000B78F4
:1031E0001342FCD17047C046000400400018004064
:1031F00070B504000D784B78002B02D08023DB00E3
:103200001D434B7A002B02D080231B011D434868CD
:1032100001280FD9431E184231D102282DD902238B
:10322000002201325B009842FBD880235B011D43E2
:10323000120415430B7A002B02D080239B011D43FF
:103240000426A6401149124A4B6813401E42FBD186
:10325000104B9847A4000D4B9C466444226A80237F
:103260005B001A402A4322626146094A4B681340B8
:103270001E42FBD1084B984770BD0022D5E70004E1
:1032800080239B0018430543D4E7C0460018004044
:10329000FC070000BD2E0000FD2E000010B504004C
:1032A0000422824009480A4943680B401A42FBD174
:1032B000084B9847A400054B9C466444226A80232F
:1032C0005B0013432362044B984710BD0018004075
:1032D000FC070000BD2E0000FD2E0000F8B5040024
:1032E000042282401248134943680B401A42FBD122
:1032F000114B98470E4F0834A400E0590007000F07
:103300000E4B98470600E559ED04ED0FE459240CE7
:103310000B4B9847002D07D1012C07D92100300015
:10332000084B9847060001E00134E6403000F8BD44
:1033300000180040FC070000BD2E00002D2F0000EB
:10334000FD2E00003564000010B50400094B9847BD
:10335000A000094B9C4660448022835840210B43C7
:1033600083504031403A43581A42FCD0034B9847AF
:1033700010BDC046BD2E000000180040FD2E00000C
:1033800010B50400094B9847A000094B9C466044C7
:103390008022835840218B4383504031403A435828
:1033A0001A42FCD1034B984710BDC046BD2E000009
:1033B00000180040FD2E000070B504000D00054B04
:1033C00098472A780F2313402034A400024AA350C0
:1033D00070BDC046813300000018004010B50400E5
:1033E000064B98472034A400054BE4582407240FCB
:1033F000044B98472000044B984710BDBD2E000099
:1034000000180040FD2E0000DD32000030B5D378FA
:10341000002B35D11378802B29D01B068024640221
:10342000234354780225AC4306D19478002C20D154
:103430008024A402234341605478013C012C1CD910
:103440000D042D0CA024E4052C431C4384620D0CB8
:10345000D02424062C431C438462D478002C22D12F
:103460005B031CD59378012B1ED0416117E000232C
:10347000D7E7C024E4022343DDE70D4C2340DFE718
:1034800041600C04240CA023DB05234383620C0C55
:10349000D0231B0623438362D378002B03D15378B8
:1034A000013B012B02D930BD8161F8E78160FAE769
:1034B000FFFFFBFF10B50A00C1090023002904D15A
:1034C0004309DB0105498C4663441F242040012148
:1034D00081401800024B984710BDC04600280040AC
:1034E0000D3400007047000010B5054B9847054BA0
:1034F0009847054B9847054B9847054B984710BD93
:10350000FD300000B92E0000E53400001911000064
:10351000E5340000FEE7000010B51A4A1A4B9A4243
:1035200011D01A00194B9A420DD2194A03339B1A33
:103530009B0801339B000022134812498C58845089
:1035400004329A42FAD1134A134B9A420AD2D34315
:1035500011495B1803218B4304339B18002102C2DD
:103560009342FCD10D4AFF210D4B8B4393600D4AD2
:1035700053687F390B4353600B4B98470B4B98476D
:10358000FEE7C046F8980000000000202C02002052
:10359000040000202C020020C004002000ED00E008
:1035A0000000000000400041ED350000891B0000D4
:1035B0000300064A1268002A04D0044A1068C3189F
:1035C000136070470249014A1160F6E7E4020020E7
:1035D000C024002001204042704780239B014B60A3
:1035E00000207047012070470020704770B500260A
:1035F0000C4D0D4C641BA410A64209D1002606F008
:1036000067F90A4D0A4C641BA410A64205D170BD8F
:10361000B300EB5898470136EEE7B300EB589847F4
:103620000136F2E7DC980000DC980000DC9800002E
:10363000E098000010B5034B0100186800F060F836
:1036400010BDC0465C000020002310B59A4200D196
:1036500010BDCC5CC4540133F8E7030082189342D8
:1036600000D1704719700133F9E7000070B505000B
:10367000002910D00C1F2368002B00DAE418280062
:1036800001F0DFFF1D4A1368002B05D16360146051
:10369000280001F0D7FF70BDA34209D92168601846
:1036A0008342F3D118685B6841182160EEE713008C
:1036B0005A68002A01D0A242F9D919685818A042C4
:1036C0000BD120680918581819608242E0D110689F
:1036D0005268411819605A60DAE7A04202D90C23F7
:1036E0002B60D5E721686018824203D110685268C8
:1036F0004118216062605C60CAE7C046E8020020B1
:10370000032370B5CD1C9D43083506000C2D1ED239
:103710000C25A9421DD8300001F093FF254A1468FA
:103720002100002919D1244C2368002B03D130003B
:1037300000F04CFD20602900300000F047FD431CE4
:103740002CD10C233000336001F07CFF03E0002D0E
:10375000DFDA0C233360002070BD0B685B1B1AD4CA
:103760000B2B03D90B60CC18256003E08C420ED1E3
:1037700063681360300001F065FF200007220B3002
:10378000231D9043C31AE7D05A42E250E4E74B6846
:1037900063600C00EEE70C004968C2E70323C41C19
:1037A0009C43A042E0D0211A300000F00FFD431CE2
:1037B000DAD1C6E7E8020020EC020020F0B58BB0B9
:1037C00014001D1E129953DA802424061B191D00B3
:1037D00014002D230B702023149E03229E43462E9B
:1037E00007D03300453B59424B411099013ACB1861
:1037F000109309AB049308AB0393139B00920293BD
:10380000109B220001932B0000F022FF0700472E9F
:1038100002D1119BDB0724D5109BFB180793462E82
:1038200014D13B78302B0CD100220023200029003A
:1038300002F086FF002804D10123109A9B1A139AE4
:103840001360139B079A1B68D31807930022002369
:103850002000290002F074FF302200280DD0079BC1
:1038600009933800099B159ADB1B13600BB0F0BD60
:103870000023AFE7591C09911A70099B07999942D7
:10388000F8D8EEE7F0B52B2385B007000C000270E6
:10389000861C002901DA2D234C427B70092C23DD84
:1038A00002ABDD1D6B1E20000A21019302F032FFE6
:1038B0006B1E3031197020000A2102F045FE040011
:1038C00009280ADC023D30342C7002AB073330008B
:1038D000AB4204D8C01B05B0F0BD019DE2E72B78D8
:1038E000013533700136F0E73023E4183370B01C33
:1038F0007470EFE7F0B595B00C000A920B931A9D27
:10390000099001F01BFE036818000D9300F048FDBC
:103910000023129323680E900C930C99277E2B683A
:103920000722C90547D59B1893431A0008322A601D
:103930001A685B68A264E3640122E56CA66C6B0004
:103940005B080F935242A74B30000F9905F054F9D2
:10395000002800D006E20122A24B524230000F990B
:1039600002F0FEFE002800D0FCE10022002330001F
:10397000290002F0EBFE002803D023002D22433360
:103980001A70994D472F00D8984D032300260C9AA2
:10399000236101339A4322600B9B13AA00932100F9
:1039A0000A9B099800F0F2F9431C00D09CE001202A
:1039B000404215B0F0BD0733B6E780236268DB00F4
:1039C000511C45D1073262600C9A0021134312AAA0
:1039D000059211AA0392232223600691019308A95C
:1039E000636852180292009332002B0004970998E2
:1039F000FFF7E4FE20233A0005009A43472A07D147
:103A0000119BDA1C02DB626893425BDD023FFFB26E
:103A10001199652F3BD8200001393A00503011919F
:103A2000FFF730FF129A060083182361012A02DC97
:103A30002268D20701D501332361232308AA9B18EA
:103A40001B78002BA8D023002D2243331A70A3E744
:103A5000672F01D0472FB7D1002A16D00C9908A89C
:103A60000B430021069112A9059111A9039123216D
:103A700009182360019300922B00049702913200F1
:103A80000998FFF79BFE0500BAE701229BE7662F26
:103A900019D1636800290CDD2161002B02D1226855
:103AA000D20702D501335B182361119B0026A36561
:103AB000C3E7002B03D101222168114200D09A1CD8
:103AC0002261F2E76727119B1298834205DB226887
:103AD0002361D207E9D50133E6E70122002B01DC9F
:103AE0009218D21A1218EBE72268530508D42369FA
:103AF0002A000A9909980B9DA847431C29D156E72B
:103B0000652F00D8DCE0A06CE16C0022002302F0FD
:103B100017FE002835D00123354A0A9909980B9DD4
:103B2000A847431C00D142E7119B129A934202DB43
:103B30002368DB070DD50B9D0E9B0D9A0A990998FA
:103B4000A8470025431C00D131E7129B013B9D4251
:103B50000BDB236800259B0700D5FDE0139BE06885
:103B6000984200DB25E7180023E7220001231A32E0
:103B70000A9909980B9EB047431C00D117E70135FD
:103B8000E3E7119B002B35DC0123194A0A990998B8
:103B90000B9EB047431C00D109E7119B002B05D1B8
:103BA000129B002B02D12368DB07D2D50B9E0E9B04
:103BB0000D9A0A990998B0470026431C00D1F6E6F1
:103BC000119B5B429E4201DB129B91E72200012385
:103BD0001A320A9909980B9FB847431C00D1E6E6B0
:103BE0000136EDE7FFFFEF7FD4940000D094000092
:103BF000E0940000A36D129E9E4200DD1E00002E88
:103C000035DC00230C93F343DB170F930F9BA76D59
:103C10000C9A3340FB1A9A4232DB119B129A934260
:103C20003CDB2368DB0739D4129E119AF31BB61ACA
:103C30009E4200DD1E00002E39DCF7430025FB17F5
:103C40000C93119A129B0C999B1A32000A409B1AF2
:103C50009D4200DB7DE7220001231A320A99099870
:103C60000B9FB847431C00D1A1E60135E9E73300BB
:103C70002A000A9909980B9FB847431CC1D196E6C0
:103C8000220001231A320A9909980B9FB847431C56
:103C900000D18CE60C9B01330C93B7E70E9B0D9A79
:103CA0000A9909980B9EB047431CBDD17FE6EA19DB
:103CB00033000A9909980B9DA847431CBDD176E6AD
:103CC000129B012B02DC01231A4238D001232A0067
:103CD0000A9909980B9FB847431C00D167E60E9BD1
:103CE0000D9A0A9909980B9FB847431C00D15EE6CC
:103CF000A06CE16C0022002302F022FD002808D015
:103D00000025129B013B9D420DDB22003300503207
:103D1000EFE6129B6A1C013B0A9909980B9DA84784
:103D2000431CF2D143E6220001231A320A99099872
:103D30000B9FB847431C00D139E60135E1E72A0063
:103D4000EAE72200012319320A9909980B9EB0472D
:103D5000431C00D12BE60135E368139A9B1A9D4260
:103D6000EFDBFBE632002B003000290004F044FFBB
:103D7000002800D121E6034D472F00D905E6024D6A
:103D800003E6C046DC940000D8940000F7B51500A7
:103D900001938A680B6900900C00934200DA1300CB
:103DA00022002B6043321278002A01D001332B60AD
:103DB00023689B0602D52B6802332B6006272368F5
:103DC0001F4027D0230043331B785A1E934122689B
:103DD000920630D42200019943320098089EB047E1
:103DE000431C25D0062320682A68E168034000258B
:103DF000042B03D18D1AEB43DB171D40A368226906
:103E0000934201DD9B1AED180027BD4220D100200E
:103E100010E00137E3682A689B1A9F42D2DA220039
:103E20000123193201990098089EB047431CF0D134
:103E300001204042FEBD3020E118433108702100CE
:103E40005A1C45310978A218433202331170C1E778
:103E5000220001231A3201990098089EB047431CA2
:103E6000E6D00137D1E70000F0B58BB006920A002A
:103E700043320793059004920A7E0C00109B6E2A31
:103E800000D18FE017D8632A2CD008D8002A00D19F
:103E900099E0582A54D026004236327029E0642A2C
:103EA00001D0692AF7D121681A68080623D5111DA7
:103EB0001960156825E0732A00D188E008D86F2AB8
:103EC00029D0702AE7D1202209680A43226003E042
:103ED000752A20D0782ADED122007821453211704F
:103EE0006C4A30E00E001A684236111D19601368E2
:103EF0003370012379E04906D9D5111D19600023DB
:103F0000D55E002D03DA2D23049A6D421370624BA7
:103F10000A2703932FE020681968050603D5081DBA
:103F200018600D6805E04006F9D50D68081D186099
:103F3000ADB2594B082703936F2A18D00A2716E011
:103F400045310A70544A03921A682168101D18609E
:103F50001568080622D5CB0702D520231943216016
:103F60001027002D03D1202322689A4322602300CA
:103F7000002243331A706368A360002B5CDB0422C9
:103F8000216891432160002D58D1049E002B64D0FC
:103F90002600039B42361B7833705EE04806DAD574
:103FA000ADB2D8E709681A68080605D5111D196071
:103FB000136862691A6006E04906F7D5111D196099
:103FC0001368A28A1A800023049E236154E01A68B1
:103FD000111D1960166800216268300001F026FB8F
:103FE000002801D0801B6060636823610023049A6D
:103FF000137041E02369320006990598079DA84790
:10400000431C43D0236800259B070FD4099BE0681D
:1040100098423DDA18003BE022000123193206994C
:104020000598079EB047431C30D00135E368099AD4
:104030009B1A9D42F0DBE9E7002DA9D0049E2800E1
:10404000390002F07DFA039B013E5B5C280033706F
:10405000390002F0EFF9051EF1D1082F09D12368CC
:10406000DB0706D563682269934202DC3023013EF8
:104070003370049B9B1B2361079B09AA00932100BB
:10408000069B0598FFF782FE431CB3D101204042F6
:104090000BB0F0BDF3940000E29400000FB40B4BA2
:1040A00013B51C68002C05D0A369002B02D1200099
:1040B00001F0AEF905AB049AA1682000019301F06C
:1040C00041FF16BC08BC04B01847C0465C00002085
:1040D000084B70B51C680500002C05D0A369002BA7
:1040E00002D1200001F094F92900A268200002F01A
:1040F00045F870BD5C00002070B505000E0000287A
:1041000004D08369002B01D101F082F9AB69AC685E
:10411000002B02D1280001F07BF9244B9C420FD1E7
:104120006C68A3891B0702D52369002B20D12100CD
:10413000280000F093F900281AD00120404270BDF9
:104140001B4B9C4201D1AC68EBE71A4B9C42E8D177
:10415000EC68E6E7013B0136A360002B04DAA269B4
:10416000934216DB0A2914D023685A1C2260197066
:104170003178A3680029EDD1013BA360002B0FDA51
:1041800022000A31280000F013F9431CD5D00A2080
:10419000D5E72200280000F00BF9431CE8D1CCE75A
:1041A0000A2023685A1C22601870C8E73495000062
:1041B000549500001495000010B5034B01001868D9
:1041C000FFF79AFF10BDC0465C000020002370B5C9
:1041D000064C050008002360FFF7EAF9431C03D1F1
:1041E0002368002B00D02B6070BDC046BC040020AB
:1041F0004A424A41802310B55200DB0000F002F829
:1042000010BD0000F0B51D004F4B85B01E680400C6
:104210000F000092002E05D0B369002B02D13000B0
:1042200001F0F6F8494B9C4250D17468009B022B78
:1042300005D0012B00D984E0002D00DA81E02100B7
:10424000300001F077F8616B002908D02300443377
:10425000994202D03000FFF709FA0023636300237C
:10426000A3616360A3891B0603D521693000FFF7B2
:10427000FDF9A389364A1340A381009B022B5AD033
:1042800003AB02AA2100300001F064F9A3891843AE
:10429000A081002D24D1029D2800FFF7CBF90195C4
:1042A000071E42D1029B0193AB4239D1012040420B
:1042B0000223A2891343A3810023A3602300473371
:1042C000236023610123636105B0F0BD214B9C4253
:1042D00001D1B468AAE7204B9C42A7D1F468A5E7B6
:1042E000002FD9D0B369002B02D1300001F090F833
:1042F000009B012B03D1A389009A1A43A2810820B5
:10430000A389276027616561184018D001201840F3
:104310000023984211D06D42A360A5611800D3E735
:104320000198FFF787F9071EC0D08023A289019D5D
:104330001343A381D6E70020BAE7A560C4E7A060D5
:10434000C2E701204042BFE75C0000203495000036
:104350005CF3FFFF54950000149500000EB410B5F7
:104360009DB002A9029008610B48822488604861D0
:10437000012040421FABC881084804CBA40000685C
:1043800001938C8101F0B2FC0023029A13701DB0DE
:1043900010BC08BC03B01847FFFFFF7F5C00002083
:1043A0000023C25C0133002AFBD1581E7047000075
:1043B000F8B505000E001400002804D08369002B16
:1043C00001D101F025F8224B9C422DD16C68A369E4
:1043D000A360A3891B0731D52369002B2ED0236846
:1043E0002269F7B2981A6369F6B2984205DB210098
:1043F000280000F09FFF002826D1A3680130013B70
:10440000A36023685A1C22601F706369984204D01D
:10441000A389DB071AD50A2E18D12100280000F045
:1044200089FF002812D00FE00A4B9C4201D1AC68F2
:10443000CDE7094B9C42CAD1EC68C8E721002800AF
:1044400000F00CF80028CAD0012676423000F8BDF2
:10445000349500005495000014950000364B70B55B
:104460001D6806000C00002D05D0AB69002B02D1A1
:10447000280000F0CDFF314B9C420FD16C680C231B
:10448000E25E93B219072DD4D90611D40923012075
:10449000336037331343A381404270BD284B9C42A5
:1044A00001D1AC68EBE7274B9C42E8D1EC68E6E72A
:1044B0005B0713D5616B002908D023004433994270
:1044C00002D03000FFF7D2F8002363632422A389CF
:1044D0009343A38100236360236923600823A28997
:1044E0001343A3812369002B0BD1A0218022A38930
:1044F000890092000B40934203D02100300001F06C
:1045000051F80123A289134011D00023A3606369ED
:104510005B42A361002023698342BED10C23E25E8B
:104520001306BAD540231343A3810138B5E7920798
:1045300000D46369A360EDE75C00002034950000BF
:104540005495000014950000F0B503690C6989B01A
:104550000700059100269C426DDC0B00013C1433E2
:10456000A50003935B1904930300143302935D19B0
:10457000049B28681B68591C019301F05BFF0190A4
:10458000B0422DD0039B02989C460696624608CA0C
:104590009446019A99B251431B0C534389190A0C52
:1045A0009B18079302881E0C069B89B2D2180368D9
:1045B000521A190C6B469B8BCB1A11145B181914E9
:1045C00092B21B041A43049B069104C06345DDD2DA
:1045D0002B68002B04D1029B043DAB422ED33C61DF
:1045E0000599380001F041FA002823DB0025019BE2
:1045F000029801330399019308C9028855199AB2A8
:10460000AA1A05681B0C2D0CEB1A15145B191D1446
:1046100092B21B04134308C0049B8B42ECD2029A53
:10462000A300D3181A68002A04D1029A043B9A42C4
:1046300009D33C61019E300009B0F0BD2B68002B0E
:10464000CDD1013CC7E71A68002AF2D1013CECE762
:10465000F0B516001F00446A9DB00490259D069693
:104660000797002C08D11020FEF7E4FF049B586246
:10467000446084600460C460049B5B6A196800291C
:104680000BD05A68012393404A608B60049801F074
:1046900012F80022049B5B6A1A60079B002B1FDA4A
:1046A00001232B607B005B080793079CB74B22001C
:1046B00019931A409A4216D1B54B249A1360069B5F
:1046C000002B03D1240301D100F091FDB14B269AB8
:1046D0000A93B14B002A01D000F08FFD00F08FFD4E
:1046E00000232B60E1E7069E079F00220023300095
:1046F000390002F025F8051E0ED00123249A13601C
:10470000A64B269A0A93002A01D100F078FDA44A0C
:1047100026990A6000F073FD1AAB01931BAB00935E
:1047200032003B00049801F01DFA630005905B0D18
:1047300000D17FE03A039B4C120B144321009A4AAC
:10474000300018959E180022984B03F03FFF984ABE
:10475000984B03F0BBFC984A984B02F073FD0400A1
:1047600030000D0004F09CFA954A964B03F0AEFC25
:1047700002000B002000290002F064FD04000D007F
:1047800004F05AFA0022039000232000290001F0CF
:10479000DDFF00280ED0039804F082FA0B0002001F
:1047A0002900200001F0CCFF030058425841039B30
:1047B0001B1A039301231693039B162B0FD88249D0
:1047C000DB00C91808684968069A079B01F0D2FF08
:1047D00000284BD0039B013B0393002316931A9BA5
:1047E0009E1B00230B933300013B0C9304D5012344
:1047F0009B1B0B9300230C93039B002B38DB039A2A
:104800000C9B944663440C9300230F920893229BC5
:104810000125092B00D991E0052B02DD0025043B81
:104820002293229B981E032800D991E001F0F8FD05
:10483000828429761A9B1B9A9E18644BF218202AB0
:104840000FDD634B0698F318D84040239B1A9C4019
:10485000204304F067FA01235E4C013E09191893C6
:1048600071E7202306989B1A9840F2E71690B6E766
:104870000B9B039A9B1A0B935342089300230F93AD
:10488000C5E701230E93239B002B65DD1F000D93CD
:10489000049A546A00226260043211001431994271
:1048A0005FD96168049800F0CEFE049B20605B6ACB
:1048B0001B680A930E2F00D905E1002D00D102E1FB
:1048C000069B079C14931594039B002B00DC85E04A
:1048D0001A000F213C4B0A40D2009B185C681B68F1
:1048E00010931194039B02241D11EB060AD53A4B39
:1048F0000D401A6A5B6A1498159902F0B3FF06908E
:1049000007910134344E002D30D1109A119B069836
:10491000079902F0A7FF069007917AE00123239AF6
:104920000E939446039B63445F1C0D933B1EAFDCC8
:104930000123ADE70023A5E70023F0E700230E9550
:104940002293013B00220D931F00133323929FE714
:1049500001230E93023BF5E701230D931F001A007C
:10496000F4E7616852000131616096E701231D425E
:1049700008D010981199E4183268736803F0A6FB08
:10498000109011916D100836BDE7C0460000F07F11
:104990000F2700000D95000010950000E094000026
:1049A000E19400000000F03F01FCFFFF0000F83F31
:1049B00061436F63A787D23FB3C8608B288AC63F25
:1049C000FB799F501344D33FA095000032040000B0
:1049D00012040000000010FE78950000039B0224E2
:1049E000002B16D0149815995D420F23CA4A2B400C
:1049F000DB00D3181A685B6803F068FB002306909D
:104A00000791C64E2D11002D00D08CE0002B00D058
:104A100081E7169B002B00D191E0069A079B10922C
:104A20001193109811990022BD4B01F08FFE0028C0
:104A300000D184E0002F00D181E00D9B002B3EDDF2
:104A400010981199039B00225E1EB64B03F03EFBAB
:104A5000069007910D9D0134200004F021F9069A7B
:104A6000079B03F033FB0022AF4B02F0EBFB1290ED
:104A70001391129B139CAD4A10931194139B9C1895
:104A80001194002D5ED1069807990022A84B03F0DF
:104A90009DFD109A23000690079101F06BFE0028FF
:104AA00000D001E3A3481399844661440B000698A3
:104AB0000799109A01F04AFE002800D0E8E2149B02
:104AC000159C069307941B9B002B00DA57E1039A71
:104AD0000E2A00DD53E1904BD2009B185C681B68E6
:104AE00008930994239B002B00DBCEE0002F00DD10
:104AF000CBE000D0CFE20898099900228C4B03F05C
:104B0000E5FA069A079B01F03FFE3E000897002851
:104B100000D0A4E20A9B0A9A5D1C31231370039B08
:104B2000013303939FE20122154205D0A418326895
:104B3000736803F0CBFA01236D10083663E7039E18
:104B40003D0089E70A9A691E521917920E9A724B14
:104B5000C900002A4AD05B181A685B6800207649B1
:104B600002F080FE109A119B03F030FD0A9B10901A
:104B7000119112930698079904F05EF8040004F06E
:104B80008FF802000B000698079903F01FFD129B97
:104B900030345D1C1C70109A119B0690079101F037
:104BA000D5FD002865D1069A079B00205C4903F0DB
:104BB0000DFD109A119B01F0C9FD002800D0BEE048
:104BC000179B9D4200D17AE7109811990022554B0E
:104BD00003F07CFA00221090119106980799514B2E
:104BE00003F074FA129506900791C3E75918086804
:104BF0004968109A119B03F069FA109011910A9C70
:104C0000179D0698079904F017F8129004F048F8D9
:104C100002000B000698079903F0D8FC129B06903F
:104C2000079130332370179B01340022A34224D113
:104C3000414B1098119902F005FB02000B000698F9
:104C4000079901F097FD002800D078E0109A119B99
:104C50000020394903F0BAFC02000B0006980799BE
:104C600001F074FD002800D129E76B1E1A78302A64
:104C700001D003963FE01D00F7E706980799294BFE
:104C800003F024FA06900791BBE70A9E089A099B55
:104C90000698079902F0E6FD03F0CEFF040003F04A
:104CA000FFFF089A099B03F011FA0B000200069817
:104CB000079903F08BFC2300303333700A9B751C7B
:104CC000EB1A9F424CD102000B0002F0BBFA060027
:104CD0000F0002000B000898099901F037FD002829
:104CE0002CD10898099932003B0001F029FD0028D9
:104CF00001D0E30722D40599049800F0DCFC0023DE
:104D00002B70039B249A01331360269B002B00D148
:104D100075E21D6073E2C046A09500007895000022
:104D20000000F03F0000244000001C400000C0FCD8
:104D3000000014400000C07C0000E03F039E6B1E9A
:104D40001A78392A06D10A9A9A4207D13023137069
:104D5000130001361A7801321A708AE71D00EEE757
:104D60000022CF4B03F0B2F90022002306900791F6
:104D70002E0001F0E5FC002800D187E7BBE70E9A82
:104D8000002A00D187E0229A012A6EDC189A002AB4
:104D900067D0C44A9B18089D0B9C0B9A0121D2181E
:104DA0000B920C9A0498D3180C9300F022FD060085
:104DB000002C0EDD0C9B002B0BDD0C9A2300944283
:104DC00000DD13000B9AE41AD21A0B920C9AD31A34
:104DD0000C93089B002B1ED00E9B002B5FD0002D48
:104DE00011DD31002A00049800F09CFD059A0100B5
:104DF0000600049800F006FD05991090049800F054
:104E00005AFC109B0593089B5A1B04D005990498E3
:104E100000F088FD05900121049800F0EAFC0F9B4A
:104E20000890002B3DDD1A000100049800F07AFD87
:104E3000229B08900025012B3BDC0025069BAB4202
:104E400033D1079B1B03AB422FD1199B079A134207
:104E50002BD00B9B013501330B930C9B01330C932F
:104E600023E036231A9A9B1A95E7089B7D1EAB42D6
:104E700006DB5D1B002F0BDA0B9BDC1B00238CE792
:104E8000089B0895EA1A0F9B00259B180F93F1E7E2
:104E90000B9C3B0081E7089D0B9C0E9E88E7089ABF
:104EA000B4E7229B0025012BC7DD0F9B0120002BBF
:104EB0000BD0089B089A1B690F9303339B00D318F0
:104EC000586800F04DFC2023181A0C9BC0181F23B3
:104ED000184000D1ABE001331B1A042B00DC9BE02F
:104EE0001C23181A0B9B24181B180B930C9B1B18C4
:104EF0000C930B9B002B05DD1A000599049800F01C
:104F000063FD05900C9B002B05DD1A0008990498A1
:104F100000F05AFD0890169B002B00D189E00899FB
:104F2000059800F0A2FD002800DB82E0039B0A2226
:104F3000013B039305990023049800F0D5FB0E9BD9
:104F40000590002B00D15DE1002331000A22049876
:104F500000F0CAFB0D9B0600002B02DC229B022BFB
:104F60006DDC002C05DD31002200049800F02CFDE2
:104F700006003000002D11D07168049800F063FB2A
:104F80003100040033690C319A1C92000C30FEF79A
:104F90005BFB01222100049800F016FD0D9F0A9B87
:104FA000013F0B93DB19370006000F930899059812
:104FB000FFF7CAFA39000D900400059800F055FD7E
:104FC00032000E900899049800F068FD01230C93BC
:104FD000C36830340500002B04D10100059800F0AF
:104FE00044FD0C902900049800F065FB0C9B229A6C
:104FF000134300D089E0069A0133134200D084E0C5
:10500000392C00D1A3E00E9B002B01DD0D9C313427
:105010000B9B5D1C1C7027E0042B00D169E70B9AE9
:105020001C33D2180B920C9AE418D31860E70300D3
:10503000F5E7002F3CDC229B022B39DD0D970D9B01
:10504000002B0CD108990522049800F04DFB089024
:105050000100059800F009FD002800DD5AE5239BBA
:105060000A9DDB43039300270899049800F023FB73
:10507000002E00D13FE6002F05D0B74203D0390003
:10508000049800F018FB3100049800F014FB32E69D
:1050900008952E00E3E7002308931E00DFE7C046D3
:1050A0000000244033040000039608952E0031E5EB
:1050B0000E9B0D97002B00D053E70A9D0899059889
:1050C000FFF742FA0A9B30300D9A28700135040030
:1050D000EB1A9A4278DC151E00DC012500270A9B9A
:1050E0005D1905990122049800F06EFC089905905D
:1050F00000F0BBFC00282FDC01D1E3072CD46B1E91
:105100001A78302AB0D11D00F9E70E9B002B07DB7F
:105110001D00229B1D4326D10123069A134222D152
:105120000C9B002B00DC73E705990122049800F02A
:105130004BFC0899059000F098FC002804DC00D096
:1051400066E7E30700D463E7392C00D05EE70B9BEA
:105150000B9A5D1C392313706B1E1A78392A3BD0C9
:1051600001321A7080E70B9B01330D930C9B002BCF
:1051700005DD392CEBD00D9D01340B9B4AE70B9BD1
:105180000F9A0D9D1C709342ABD000230A22059903
:10519000049800F0A9FA002305900A223900049827
:1051A000B74206D100F0A0FA070006000D9B0B9352
:1051B000FCE600F099FA3100070000230A22049867
:1051C00000F092FA0600F1E700230A2205990498FC
:1051D00000F08AFA059071E70A9A9A4205D1039B7A
:1051E00001330393312313703EE71D00B4E70A4BEC
:1051F000269A0A93094B002A01D0269A13600A982E
:105200001DB0F0BD0D9B002B00DD56E7229B022B4D
:1052100000DC52E713E7C046049500000C9500003F
:10522000F7B58A8905000C00130760D44B68002B82
:1052300004DC0B6C002B01DC0020FEBDE76A002FB4
:10524000FAD000232E682B6080235B011A4034D0F3
:10525000606DA3895B0706D56368C01A636B002B7A
:1052600001D0236CC01A0200216A00232800E76ADB
:10527000B847A189431C06D12B681D2B31D82C4A75
:10528000DA40D3072DD50023636023692360CB0464
:1052900005D5431C02D12B68002B00D16065616BE2
:1052A0002E600029C8D023004433994202D0280040
:1052B000FEF7DCF900206063BFE70123216A2800C4
:1052C000B847431CC5D12B68002BC2D01D2B01D081
:1052D000162B01D12E60AFE74023A2891343A3818F
:1052E000ABE740230B430120A3814042A5E70F69B0
:1052F000002FA1D00B680F60DB1B019300239207E6
:1053000000D14B69A360019B002B00DC94E7019B5B
:105310003A00216A2800A66AB047002803DC40232F
:10532000A2891343DFE7019B3F181B1A0193EAE7A9
:10533000010040200B6970B505000C00002B01D165
:10534000002070BD002804D08369002B01D100F03B
:105350005FF80B4B9C4209D16C680C22A35E002BBA
:10536000EED021002800FFF75BFFEAE7054B9C42E7
:1053700001D1AC68F1E7044B9C42EED1EC68ECE75C
:1053800034950000549500001495000010B50249B2
:1053900000F0B2F810BDC04635530000002310B530
:1053A000040003604360836081814366C2810361BE
:1053B00043618361190008225C30FEF74EF9054B0A
:1053C00024626362044BA362044BE362044B2363D5
:1053D00010BDC046E9610000116200004962000092
:1053E0007562000070B568254A1E55430E002900FD
:1053F0007431FEF785F9041E08D000212A000160EF
:1054000046600C30A0606832FEF727F9200070BDBE
:10541000836913B50400002B28D18364C36403653A
:10542000134B144A1B6882620193984201D10123F5
:105430008361200000F020F86060200000F01CF87C
:10544000A060200000F018F80022E06004216068ED
:10545000FFF7A4FF01220921A068FFF79FFF0222A6
:105460001221E068FFF79AFF0123A36113BDC04634
:10547000CC9400008D530000F8B51E4B07001E6849
:10548000B369002B02D13000FFF7C2FF4836B46881
:105490007368013B04D53368002B07D03668F6E704
:1054A0000C22A55E002D0DD06834F2E704213800EF
:1054B000FFF798FF30600028F0D10C2304003B6018
:1054C0002000F8BD012320005B42E3810233A38169
:1054D00065662560A560656025616561A561082236
:1054E00029005C30FEF7B9F86563A563A564E5643F
:1054F000E6E7C046CC940000F7B50400070000269C
:1055000001914834002C01D13000FEBD6368A568CC
:105510000093009B013B009301D52468F2E7AB891F
:10552000012B08D90E22AB5E013304D029003800CC
:10553000019B984706436835EBE70000034B1B6867
:10554000186A002800D10248F03070475C00002043
:10555000C000002070B50E001D000E23C95E90B083
:105560001400002907DA00232B60B3891B0611D42D
:105570008023DB000FE001AA00F0A8FE0028F2DB88
:10558000F022029B12021340054A9B185A425341D3
:105590002B60EDE740230020236010B070BDC046B3
:1055A00000E0FFFFF7B502268B8905000C003342AF
:1055B00006D0230047332360236101236361F7BDD5
:1055C00001AB6A46FFF7C6FF009907002800FEF707
:1055D00097F8002808D10C22A35E9A05EFD4032285
:1055E00093431E43A681E4E70F4BAB628023A2895D
:1055F00020601343A381009B20616361019B002B0A
:105600000DD00E23E15E280000F072FE002806D0C7
:105610000322A38993431A0001231343A381A08982
:105620003843A081CBE7C0468D530000C9B2821831
:10563000904201D10020704703788B42FBD00130AB
:10564000F6E77047704770B5466A04000D00002EFB
:1056500007D11020FDF7EEFF6062466086600660AD
:10566000C660666AF368002B13D0636AAA00DB6821
:105670009B181868002818D101210E00AE40721D39
:105680009200200000F0C2FA00280CD0456086602D
:105690000DE021220421200000F0B8FA636AF060D6
:1056A000DB68002BE1D1002070BD02681A60002386
:1056B0000361C360F8E770B5446A06000D00002C72
:1056C00007D11020FDF7B6FF70624460846004606B
:1056D000C460002D07D0736A6A68DB6892009B186B
:1056E0001A682A601D6070BDF7B51E0014239C4621
:1056F00007000C0000200D698C44634619881B6864
:1057000051431B0C534389190E0C9B1989B21E0C73
:105710001B045B186146013008C18C468542ECDCF5
:10572000002E1BD0A3689D4212DB63683800591C11
:10573000FFF789FF2100236901909A1C92000C3128
:105740000C30FDF781FF21003800FFF7B4FF019C0A
:105750002B1D9B00E31801355E6025612000FEBD16
:105760000300020C0020824201D11B0410301A0EEB
:1057700001D108301B021A0F01D104301B019A0F0E
:1057800001D102309B00002B03DB01305B0000D411
:10579000202070470722036810B501001A400DD081
:1057A00001240020234205D10230034203D0E3400C
:1057B00020000B6010BD9B080B60FBE79CB2100043
:1057C000002C01D110201B0CDAB2002A01D10830C4
:1057D0001B0A1A0701D104301B099A0701D10230B4
:1057E0009B08DA07E8D45B0801D00130E4E7202009
:1057F000E0E710B50C000121FFF725FF012344610C
:10580000036110BDF0B50B691500126989B00C0079
:10581000934201DA2C000D0027692E69A268BB199A
:1058200061680193934200DD0131FFF70CFF030033
:1058300014330093009ABB1994469B009C441300B8
:105840000022049063451CD32A001434BF00E319DE
:105850001432B6000593931902940693069B9A425C
:1058600011D3019B002B06DD04235B429C4463465D
:105870001B68002B51D0049B019A18001A6109B0D3
:10588000F0BD04C3DEE71488002C1ED00026009D66
:10589000029F01CF079508CD039383B2634319009C
:1058A0006B46000C9B896043CB1803999B19090C2C
:1058B0004118180C09180E0C9BB209040B430799E8
:1058C0000B60059BBB42E4D82E6013681B0C03934E
:1058D0001ED00026009B029C1B68009807002188B0
:1058E000039D9BB2694320C82D0C49198E193104C0
:1058F0000B433B6008CC03991B0C4B437968360C77
:1059000089B25B1805999B191E0CA142E6D8036069
:10591000009B043204330093A0E7019B013B0193F9
:105920009FE700000323F7B5134005000E001400A5
:10593000002B08D02249013B9A0052580023310025
:10594000FFF7D2FE0600A310019336D06C6A002C3C
:1059500007D11020FDF76EFE686244608460046029
:10596000C4606F6ABC68002C07D116492800FFF795
:1059700040FF00230400B86003600122019B134232
:105980000AD0310022002800FFF73CFF0700310059
:105990002800FFF790FE3E00019B5B1001930CD0A6
:1059A0002068002807D1220021002800FFF72AFFE5
:1059B0000023206003600400DFE73000FEBDC04626
:1059C0006896000071020000F0B50D0017002B6909
:1059D000541185B0E3180293013301934968AB6811
:1059E0000390019A934234DB0398FFF72CFE0023C7
:1059F0000200060019001432A3422DDBE343DB173B
:105A00001C402B001F21A40014192A691433920092
:105A10009A180F4024D00131C91B8C460021186808
:105A2000B84001436046216002CB0434C1409A4231
:105A3000F5D82160002902D0029B02330193019B1B
:105A40000398013B33612900FFF735FE300005B0B4
:105A5000F0BD01315B00C4E7980011500133CBE782
:105A600002CB02C49A42FBD8E9E70A69036930B560
:105A70009B1A0ED192001430143184188918043CFA
:105A8000043922680D68AA4205D0AA429241012336
:105A90001343180030BDA042F1D3FAE7F0B50D0072
:105AA00085B00700110028001400FFF7DEFF061E76
:105AB00008D101003800FFF7C6FD012346610361EC
:105AC00005B0F0BD01230193002804DB23002C0066
:105AD0001D000023019361683800FFF7B4FD2F001B
:105AE0000022019B2669C3601434B300E3180293BB
:105AF0002B6914379B00FB1803930300944614335F
:105B000020CC04CF0192AAB294446A46614692889E
:105B10002D0C8A1A0199090C691A151449190D14CA
:105B200092B209040A431A60039AAC460433BA429B
:105B3000E6D802991A008C4205D3043A1368002B68
:105B40000ED00661BCE704CC91B261440D14120C76
:105B50005219151489B212040A43AC4604C3E8E78B
:105B6000013EEAE7F7B51D000121089F1400FFF789
:105B70006AFD2B036D0006001B0B6D0D24D10193F4
:105B8000002C27D068460094FFF704FE009C0028F4
:105B90001ED0019B20211A00091A8A40C3402243CB
:105BA00072610193019CB461631E9C4101343461B4
:105BB000002D18D0124BED1835232D183D60181A02
:105BC000099B18603000FEBD802252031343D6E7C4
:105BD0007461E7E701A8FFF7DDFD0124019B346153
:105BE00073612030E4E7074BC018074B3860E318B7
:105BF0009B00F3185869FFF7B3FD6401201ADFE733
:105C0000CDFBFFFFCEFBFFFFFFFFFF3F4A4370B519
:105C100011001400FDF774FD051E03D022000021C1
:105C2000FDF71BFD280070BDF0B58E6885B007003C
:105C30000C00039201939E4239D890238A89DB009D
:105C40001A4234D00325096923685B1A02936369F9
:105C500002985D43EB0F5D19019B6D1001331B181A
:105C6000AB4200D91D00530532D529003800FDF79D
:105C700047FD061E09D10C233B6040230120A28969
:105C800040421343A38105B0F0BD029A2169FDF79C
:105C9000DBFCA389144A1A4080231343A381029B8F
:105CA0002661F61826606561019EED1AA560019BCC
:105CB000B34200D21E0032000399206800F050FB6E
:105CC000A36800209B1BA36023689E192660DAE767
:105CD0002A00380000F056FB061EE0D1216938008A
:105CE000FDF7C4FCC7E7C0467FFBFFFFF0B59FB0E0
:105CF000029005938B890F0016001B0611D50B69C6
:105D0000002B0ED14021FDF7FBFC386038610028E4
:105D100005D10C23029A013813601FB0F0BD402357
:105D20007B61002306AD6B6120336B761033AB765D
:105D300034002378002B47D1A31B04930DD0A31B61
:105D4000320039000298FFF76FFF431C00D1B5E025
:105D50006A69049B944663446B612378002B00D1ED
:105D6000ACE00122002352426A6002A95432521868
:105D700001342B60EB60AB601370AB65584E0522AD
:105D800021783000FFF752FC621C002820D12968DE
:105D9000CB0604D5532302AE20309B1918700B0795
:105DA00004D553232B2002AE9B19187023782A2B7D
:105DB00016D000200A21099B2278303A092A55D9A9
:105DC000002815D0099313E0252BB5D00134B0E796
:105DD0000123801B8340296814000B432B60CDE70F
:105DE000059B181D1B680590002B39DB09931400D7
:105DF00023782E2B0BD16378621C2A2B3ED1059B76
:105E000002341A1D1B680592002B34DB0793354EB4
:105E1000217803223000FFF709FC002806D0402338
:105E2000801B83402A68013413432B6021780622AB
:105E30002D48661C2976FFF7F9FB002846D02B4B2E
:105E4000002B2FD12968059B0722C90528D59B184F
:105E50009343083305936B69039A9B186B6167E75B
:105E60005B42EB6002230B432B60C0E74B430134E2
:105E70009B180120A0E701235B42C7E70023140021
:105E80000A201A006B6021783039092903D9002BC8
:105E9000BDD00792BBE74243013452180123F2E719
:105EA0000733D5E705AB00933A00114B2900029860
:105EB000FDF720FD0390039B0133CCD1BB890B98E8
:105EC0005B0600D429E70120404226E705AB00939A
:105ED0003A00074B29000298FDF7C6FFEAE7C046E3
:105EE000749600007A9600007E960000F538000057
:105EF000295C0000936810B5013B9360002B05DA24
:105F00009469A34208DBCBB20A2B05D01368581C56
:105F100010601970C8B210BDFEF74AFAFBE7F8B579
:105F200006000F001400D518AC4201D1002007E094
:105F300021783A003000FFF7DDFF0134431CF3D134
:105F4000F8BD0000F0B59FB006000F0014000593E7
:105F5000002804D08369002B01D1FFF759FA7F4B49
:105F60009F425CD17768BB891B0762D53B69002BD8
:105F70005FD0002306AD6B6120336B761033AB76B8
:105F80000294029C2378002B5DD1029BE31A0493B8
:105F90000DD0049B029A39003000FFF7C0FF431C6C
:105FA00000D1CCE06A69049B944663446B6123781A
:105FB000002B00D1C3E00122002352426A6002A9F3
:105FC0005432521801342B60EB60AB601370AB6538
:105FD000217805226248FFF729FB631C9C460028B4
:105FE00035D12968CB0604D5532302AA20309B184B
:105FF00018700B0704D553232B2002AA9B18187086
:1060000023782A2B2CD000200A21099B2278303AB1
:10601000092A00D86BE000282AD0099328E0514BC8
:106020009F4201D1B7689EE74F4B9F429BD1F768D3
:1060300099E739003000FEF711FA002899D00120C5
:1060400040421FB0F0BD252B9FD001349AE7444B4E
:106050002968C01A012383400B432B606446B7E7CD
:10606000059B181D1B680590002B3ADB09936446BD
:1060700023782E2B0BD16378621C2A2B3FD1059BF2
:1060800002341A1D1B680592002B35DB079321781B
:1060900003223648FFF7CAFA002807D0334B2A6894
:1060A000C01A4023834013432B6001342178631CC2
:1060B00006222F4802932976FFF7B8FA002844D029
:1060C0002C4B002B2FD12968059B0722C90528D509
:1060D0009B189343083305936B69039A9B186B6174
:1060E0004FE75B42EB6002230B432B60BFE74B4360
:1060F00001349B18012089E701235B42C6E7002396
:1061000014000A201A006B6021783039092903D95C
:10611000002BBCD00792BAE7424301345218012346
:10612000F2E70733D5E705AB00933A00124B29009D
:106130003000FDF7DFFB0390039B0133CCD1BB891B
:106140005B0600D57BE70B987BE705AB00933A0035
:10615000094B29003000FDF787FEECE7349500007D
:106160007496000054950000149500007A96000083
:106170007E960000F53800001F5F000070B5060035
:106180000D001400002804D08369002B01D1FFF713
:106190003FF9124B9C4211D17468A368013BA36084
:1061A000002B05DAA269934212DBEBB20A2B0FD067
:1061B0002368E8B25A1C22601D7070BD084B9C42D7
:1061C00001D1B468E9E7074B9C42E6D1F468E4E703
:1061D000220029003000FEF7EBF8EEE734950000CE
:1061E000549500001495000070B50C000E25495F11
:1061F00000F0EEF8002803DB636D1B18636570BDCB
:10620000A389024A1340A381F9E7C046FFEFFFFFCD
:10621000F8B51F008B8905000C001600DB0505D5BD
:106220000E23C95E0022022300F074F8A389054AF8
:1062300028001340A38132000E23E15E3B0000F0F2
:106240001FF8F8BDFFEFFFFF70B50C000E25495F8A
:1062500000F060F8A389421C03D1054A1340A381D2
:1062600070BD802252011343A3816065F8E7C046E8
:10627000FFEFFFFF10B50E23C95E00F015F810BD4B
:1062800070B50500080011000022064C22601A00BB
:10629000FBF796F9431C03D12368002B00D02B6039
:1062A00070BDC046BC040020002370B5064C05003C
:1062B00008002360FDF78EF9431C03D12368002BEF
:1062C00000D02B6070BDC046BC040020002370B518
:1062D000064C0500080011002360FDF77EF9431C01
:1062E00003D12368002B00D02B6070BDBC040020BC
:1062F000002370B5064C050008002360FDF772F915
:10630000431C03D12368002B00D02B6070BDC04616
:10631000BC04002070B50500080011000022064CE6
:1063200022601A00FDF760F9431C03D12368002B9B
:1063300000D02B6070BDC046BC04002082B0002994
:1063400000D101A9101E06D0002B06D013780B60D7
:106350001078431E984102B0704702204042FAE78D
:1063600010B5884202D98B18984208D300239A426C
:1063700007D0CC5CC4540133F9E78B5C8354013AF9
:10638000FBD210BDF8B507000D001600002905D19D
:106390001100FDF7B5F904002000F8BD002A03D173
:1063A000FDF764F93400F7E700F032F82C0086427C
:1063B000F2D931003800FDF7A3F9041EECD0290012
:1063C0003200FDF741F929003800FDF74FF9E3E706
:1063D00070B50500080011000022064C22601A006A
:1063E000FBF7CCF8431C03D12368002B00D02B60B3
:1063F00070BDC046BC0400200B1E04D0FF2A04D987
:106400008A2303608B3B180070470A700123FAE768
:106410000B1F1B68181F002B01DA0B58C0187047A0
:1064200002B4714649084900095C49008E4402BC27
:106430007047C046002243088B4274D303098B4245
:106440005FD3030A8B4244D3030B8B4228D3030C44
:106450008B420DD3FF22090212BA030C8B4202D3E6
:106460001212090265D0030B8B4219D300E0090A0E
:10647000C30B8B4201D3CB03C01A5241830B8B4217
:1064800001D38B03C01A5241430B8B4201D34B0300
:10649000C01A5241030B8B4201D30B03C01A524165
:1064A000C30A8B4201D3CB02C01A5241830A8B42EA
:1064B00001D38B02C01A5241430A8B4201D34B02D3
:1064C000C01A5241030A8B4201D30B02C01A524137
:1064D000CDD2C3098B4201D3CB01C01A52418309EB
:1064E0008B4201D38B01C01A524143098B4201D325
:1064F0004B01C01A524103098B4201D30B01C01A50
:106500005241C3088B4201D3CB00C01A52418308C9
:106510008B4201D38B00C01A524143088B4201D3F6
:106520004B00C01A5241411A00D201465241104656
:106530007047FFE701B5002000F0F0F802BDC0464B
:106540000029F7D076E7704703460B437FD400223B
:1065500043088B4274D303098B425FD3030A8B42F7
:1065600044D3030B8B4228D3030C8B420DD3FF2261
:10657000090212BA030C8B4202D31212090265D02F
:10658000030B8B4219D300E0090AC30B8B4201D3E2
:10659000CB03C01A5241830B8B4201D38B03C01A29
:1065A0005241430B8B4201D34B03C01A5241030BA0
:1065B0008B4201D30B03C01A5241C30A8B4201D351
:1065C000CB02C01A5241830A8B4201D38B02C01AFC
:1065D0005241430A8B4201D34B02C01A5241030A73
:1065E0008B4201D30B02C01A5241CDD2C3098B4258
:1065F00001D3CB01C01A524183098B4201D38B01D5
:10660000C01A524143098B4201D34B01C01A524177
:1066100003098B4201D30B01C01A5241C3088B42BC
:1066200001D3CB00C01A524183088B4201D38B00A7
:10663000C01A524143088B4201D34B00C01A524149
:10664000411A00D201465241104670475DE0CA0F20
:1066500000D04942031000D34042534000229C46E0
:1066600003098B422DD3030A8B4212D3FC228901EA
:1066700012BA030A8B420CD3890192118B4208D3C0
:10668000890192118B4204D389013AD0921100E022
:106690008909C3098B4201D3CB01C01A5241830936
:1066A0008B4201D38B01C01A524143098B4201D363
:1066B0004B01C01A524103098B4201D30B01C01A8E
:1066C0005241C3088B4201D3CB00C01A5241830808
:1066D0008B4201D38B00C01A5241D9D243088B425E
:1066E00001D34B00C01A5241411A00D20146634601
:1066F00052415B10104601D34042002B00D5494265
:10670000704763465B1000D3404201B5002000F0A3
:1067100005F802BD0029F8D016E770477047C0465B
:106720008446101C62468C46191C634600E0C04635
:106730001FB501F069FC002801D40021C8421FBD2B
:1067400010B501F0C3FB4042013010BD10B501F09F
:106750005BFC002801DB002010BD012010BDC046FD
:1067600010B501F051FC002801DD002010BD012012
:1067700010BDC04610B501F0E3FB002801DC00208D
:1067800010BD012010BDC04610B501F0D9FB002896
:1067900001DA002010BD012010BDC046002B11D130
:1067A000002A0FD1002900D1002802D00021C943BE
:1067B000081C07B4024802A14018029003BDC0465D
:1067C0005DFFFFFF03B4684601B5029800F030F8A2
:1067D000019B9E4602B00CBC7047C046F0B5CE4649
:1067E000474615042D0C2E0080B50704140C3F0CF1
:1067F0009946030C7E435D43674363437F19340C22
:10680000E4199C46A54203D980235B029846C44400
:106810004B46514343433604360C250C240465444F
:10682000A4195918491920000CBC90469946F0BD8E
:10683000F0B557464E464546DE46E0B5040083B007
:106840000D00924699468B422FD82CD0494650468F
:1068500002F010FB29000600200002F00BFB331AA7
:106860009846203B9B4600D574E053465A469340D9
:106870001F005346424693401E00AF4229D826D0FF
:106880005B46A41BBD41002B00DA79E00022002307
:106890000092019301235A469340019301234246FB
:1068A0009340009319E08242D0D900220023009245
:1068B00001930C9B002B01D01C605D600098019936
:1068C00003B03CBC90469946A246AB46F0BDA342FD
:1068D000D6D900220023009201934346002BE8D032
:1068E000FB0772081A4346467B080EE0AB4201D113
:1068F000A2420CD8A41A9D41012024196D41002107
:10690000013E24184D41002E06D0AB42EED9013E87
:1069100024196D41002EF8D15B46009801990019A9
:106920006941002B22DB2B005A46D3402A00444603
:10693000E2401C005B461500002B2CDB26009E402D
:10694000330026004746BE403200801A994100902D
:106950000191AEE7424620239B1A5246DA40414657
:1069600013004A468A4017001F4382E7424620230D
:106970009B1A2A0046469A402300F3401343D5E76A
:106980004246202300219B1A0022009101920122FD
:10699000DA40019282E74246202326009B1ADE401D
:1069A0002F00B446974066463B003343C9E7C046D4
:1069B000F0B557464E46DE464546E0B54402430034
:1069C000C60F83B00F1C640A1B0EB24653D0FF2BB8
:1069D00027D08022E400D20414437F225242904602
:1069E0009844002399469B467D027800FB0F6D0A70
:1069F000000E009324D0FF2846D080230021ED0014
:106A0000DB041D437F384746381A4F460F43BF000B
:106A1000B9463300009A874F53404A46BA5801930B
:106A20009746002C4ED108239946F7339846FD3BF4
:106A30009B467D027800FB0F6D0A000E0093DAD1B1
:106A4000002D26D1002001213300009A7A4F5340B7
:106A50004246101A4A460A439200BA581D00974609
:106A6000009B2C009A468B465B46022B31D1534645
:106A7000FF21002438E0002C17D10423994600237D
:106A8000984601339B46AFE7FF20002D0BD1022132
:106A9000DAE7280002F0D0F9431F9D4076235B42DD
:106AA000181A0021AFE70321ADE7200002F0C4F976
:106AB000431F9C4076235B421B1A9846002399464D
:106AC0009B4691E70C239946F3339846FC3B9B4643
:106AD0008AE7032B00D1A5E05546012B00D081E0C9
:106AE0000123002100242B406402C905600ADB0752
:106AF0000843184303B03CBC90469946A246AB46B7
:106B0000F0BD80240023E403FF21EDE7FF210024F2
:106B1000EAE70123591A1B2966DD019A1340002177
:106B20000024E1E78023DB031C4238D01D4251D012
:106B30001C436402640A3300FF21D5E763016C0142
:106B4000A3423BD21B260021013801251F0049002A
:106B50005B00002F01DB9C4201D81B1B2943013E37
:106B6000002EF3D11C00631E9C410C4301007F31B9
:106B70000029CEDD630704D00F232340042B00D06F
:106B80000434230103D501002C4B80311C40FE2925
:106B90000DDD0123019AFF2113400024A4E7802387
:106BA000DB031C436402640A3300FF219CE70123DA
:106BB000019AA401640AC9B2134095E71B1B1A2667
:106BC0000121C2E7009B8B469A4600244CE76302F2
:106BD000E5D500258024E4032C436402640A009B6D
:106BE000FF2181E70195C1E723002020CB40411A16
:106BF0008C40611E8C411C43630704D00F2323404B
:106C0000042B00D00434630105D50123019A01212E
:106C10001340002468E70123019AA401640A134089
:106C2000002161E78023DB031C436402640A5346AE
:106C3000FF2159E790970000D0970000FFFFFFF772
:106C4000F8B557464E464546DE46E0B54702460093
:106C500088467F0A360EC40F002E47D0FF2E24D060
:106C6000FB008027FF041F43002399469A467F3E7E
:106C700043465D025800DB0F6D0A000E984643D074
:106C8000FF283BD0EB0080250022ED041D437F3818
:106C90003618731C41469B464B46614013430F2BED
:106CA00064D875489B00C3589F46002F42D10823E3
:106CB0009946063BFF269A46DAE74146022A28D043
:106CC000032A00D1CEE0012A00D0ACE01140002020
:106CD0000022CCB24002D205400AE4071043204310
:106CE0003CBC90469946A246AB46F8BD002F15D154
:106CF00004239946033B00269A46B9E7FF20022267
:106D0000002DC5D00322C3E7002D19D10020012298
:106D1000BEE70124FF220C400020DBE7380002F030
:106D20008BF87626431F9F4000237642361A9946F9
:106D30009A469DE70C239946093BFF269A4697E71A
:106D4000280002F079F8431F9D4076235B42181A11
:106D500000229DE780200024C003FF22BAE73D0007
:106D60005246ABE73D0021005246A7E73B0C9C464C
:106D70002A04120C2B0C1400604665463F043F0C9D
:106D80007C4342435D437B43270C9B18FF18BA4268
:106D900003D980235B029C46654424043A04240CF6
:106DA000121993015C1EA3413F0C920E7D191A43E8
:106DB000AD0115432B0104D501235E466A081D4031
:106DC000154332007F32002A25DD6B0704D00F23E4
:106DD0002B40042B00D004352B0103D53200274B68
:106DE00080321D40FE2A94DC0124A801400AD2B260
:106DF0000C406FE78020C003074207D0054205D151
:106E000028434002400A4446FF2263E738434002D9
:106E1000400AFF225EE70124A31A1B2B05DD0C406C
:106E20000022002056E75E46CBE72A002020DA4009
:106E3000C31A9D402B005D1EAB4113435A0704D07B
:106E40000F221A40042A00D004335A0104D5012429
:106E500001220C4000203DE701249B01580A0C4010
:106E6000002237E780200124C00328434002400A63
:106E70000C40FF222EE7C04610980000FFFFFFF7EE
:106E8000F0B54F46D64646464400C0B5C20F47024D
:106E90004802400A844666467B0A4800C90F9A4663
:106EA000240E1500DB00000E8946F600FF2800D1F5
:106EB0008FE001214F464F403900914266D0221A9F
:106EC000002A00DC9DE000283DD1002E00D18BE09F
:106ED000511E002900D0B5E001249B1B5A0144D566
:106EE0009B019F09380001F0A7FF053887408442C5
:106EF00000DD96E0041B3A0020200134E240041B30
:106F0000A7403B005F1EBB41002413435A0704D037
:106F10000F221A40042A00D004335A0127D5013425
:106F2000FF2C00D179E001229B015B0AE4B22A40E8
:106F30005B02E405580AD207204310431CBC90466C
:106F40009946A246F0BDFF2CE0D08021C9040E4333
:106F50001B2A7BDC31002020D140821A9640721E11
:106F600096410E439B1B5A01BAD45A07D0D1012235
:106F7000DF082A40FF2C33D1002F00D1A8E0802366
:106F8000DB033B435B025B0AFF24D1E7211A0029A4
:106F90004CDD00282AD0FF2CB8D08020C004064346
:106FA0001B2900DDAFE030002027C840791A8E4051
:106FB000711E8E4106439B195901D6D50134FF2C11
:106FC00000D185E001227A491A405B080B40134347
:106FD0009CE7002E00D070E76BE73B1EC5D1002276
:106FE0007B025B0AE4B2A3E714008FE7002E4DD0CA
:106FF000481E002857D19B1901245A01B5D50224F7
:10700000E0E7002A25D1621CD2B2012A72DD9F1B63
:107010007A0135D5F71A0D0064E7012200232A40D2
:1070200086E73B00634A241A13406FE700296CD1BE
:10703000611CC8B201284EDDFF2949D09B195B08AD
:107040000C0063E7FF2A41D00A0081E701269B1B61
:1070500089E7002C1CD0FF2821D08024E404524270
:1070600023431B2A00DD96E01C002025D440AA1AE9
:1070700093405A1E93412343F31A04000D002DE759
:10708000002F00D02EE700220024A9E70C003DE7E6
:10709000002B58D0D243002AEED0FF28E1D1330094
:1070A000FF240D0032E7FF2910D0010078E7002B04
:1070B0006ED0FF24002E00D128E780225146D20353
:1070C000114203D06146114200D13300FF241DE775
:1070D000FF2400232CE7002CE9D1002B63D0002EE5
:1070E00000D113E79B195A0100D43EE7314A0C0046
:1070F00013400BE7002C1ED1002B2FD1002E4FD0B8
:1071000033000D0002E7012655E7002C1FD1002BAC
:1071100043D0C94300290BD0FF2839D01B2944DCB8
:107120001C002027CC40791A8B40591E8B412343E9
:107130009B19040040E7002B1AD1002E24D1802790
:107140000022FF031BE7330004000D00DEE6FF28EA
:107150001ED08024E40449422343DFE7002E00D1FF
:10716000D4E69F1B7A0100D437E7F31A0D00CDE671
:10717000FF24002E00D1C9E680225046D2031042DF
:10718000A4D060461042A1D133000D00FF24BDE61B
:107190003300FF24BAE601236EE733000400B5E6AE
:1071A000002700221CE73300B0E60123C0E7C046F9
:1071B000FFFFFF7DFFFFFFFB10B5041E27D001F08E
:1071C0003BFE9E231B1A962B0ADC9622D21A944071
:1071D0006402640ADBB26402DB05600A184310BD76
:1071E000992B17DC9922D21A002A27DD944022001D
:1071F000134C1440510704D00F210A40042A00D038
:107200000434620112D4A401640ADBB2E3E7002370
:107210000024E0E7B9222100D21A91400A00511E51
:107220008A410521091ACC401443DBE7044B1C407A
:107230009F23A4011B1A640ADBB2CCE72200D7E724
:10724000FFFFFFFBF8B54546DE4657464E460C03AA
:10725000E0B54E00C90F88460D00610A440F0C438B
:10726000C70019035800DB0F9B464B0A510F0B4315
:10727000760D400D1900D200D84500D1AEE0351A88
:10728000002D00DCF6E000280FD1134300D1DBE035
:107290006B1E002B00D037E1BA1A9742BF41641A27
:1072A0007F42E41B0126170024E0C64B9E424DD0CE
:1072B00080231B041943382D00DD07E11F2D00DD5D
:1072C00038E12020431B9A460B00504683409946E4
:1072D00013004846EB401843030050468240501EBE
:1072E0008241E9401A43BA1A611A9742A441170031
:1072F00064420C1B230262D56402650A002D00D192
:10730000DFE0280001F098FD0300083B1F2B00DDA3
:10731000D2E020223C00D21A9D40D4409F40254319
:107320009E4200DDC4E09E1B731C1F2B00DDF1E0BC
:10733000202238002900D21AD840914097402C00D2
:107340000143781E8741DC4000260F437B0709D0AC
:107350000F233B40042B05D03B1DBB42BF417F4266
:10736000E4191F0023022CD5964B01369E4200D112
:107370009AE04546944BFF081C406007760564027E
:107380000743240B760D00212403230B0C0D8F4A99
:1073900024051C431440330523435B00ED075B08C1
:1073A0002B43380019003CBC90469946A246AB4698
:1073B000F8BD6446044300D111E2040067467B0730
:1073C000C6D145466007FF080743E4087D4B9E424F
:1073D00030D024037605240B760DD4E7331A9A4671
:1073E000002B78DD002831D076488642AED0802050
:1073F000000401435346382B00DCE9E00A43511EE8
:107400008A410021D219BA42BF4109197C421700B2
:107410000C192302D3D56B4B01369E4200D13AE1C1
:107420000120694B1C407B0807401F43E0070743CE
:1074300064088BE723003B4300D1CBE18022120399
:1074400014432403240B9EE72E007FE7080010431B
:1074500000D1B4E0581E002800D0DEE0BA18BA42CD
:107460009B4164185B42E418170001262302A6D54D
:107470000226D5E7002D6ED1701C4005400D012875
:1074800000DCF9E0B81A844687428041E51A4042A0
:107490002D1A280200D489E0D71BBA4292411C1B46
:1074A0005242A51AD84629E74546002400276AE734
:1074B000454CF61A2C4049E73D0028388540002706
:1074C0002EE7380001F0B8FC20301DE70A43511EBA
:1074D0008A41002107E7002B00D0F3E0701C430530
:1074E0005B0D012B00DCADE0364B984200D1D1E0C2
:1074F000BA18BA42BF4164187F42E419E70752083C
:1075000017436408060021E72E48854200D193E026
:107510001D00D0E629001F3EF140202B00D18DE058
:107520004022D31A9D402F437D1EAF4100240F43BC
:10753000002644E72B000800203BD8400300202D04
:1075400000D17DE04020451BA9400A43511E8A41DD
:1075500000211A43C7E6002E50D01A4EB04257D031
:1075600080266B429946360434434B46382B00DD67
:10757000D6E01F2B00DD35E12026F51A2600AE40AF
:10758000B2463E00DE40AC46350056462E436546C8
:10759000AF407D1EAF41DC403743D71BBA4292411A
:1075A0000C1B5242A41A0600D846A3E6644667465E
:1075B0002C4300D0A2E600250026002706E71E0087
:1075C000C4E6C046FF070000FFFF7FFFFFFF0F80FC
:1075D0001F2B63DC2020C31A080098409C4683467A
:1075E00053461000D84003005846184363469A405B
:1075F000531E9A4153460243D94003E726003E43B7
:1076000006D0EB439946002BC7D0944EB042ACD184
:107610000C0017000600D84698E6904B9A450BD010
:107620008246E7E6002800D09EE01800104300D113
:10763000E9E01C001700D846884E87E6002572E76F
:10764000002182E723003B43002E00D0ABE0002B5B
:1076500000D1E7E00B00134300D177E6BA18BA4235
:10766000BF4164187F42E419230200D4F2E07C4B4E
:1076700017001C40060069E620003843002ED1D1D7
:1076800000285BD11C00144300D1A8E01C001700A7
:10769000D8465BE606000024002797E650460B001C
:1076A0002038C34099465346202B00D195E0402313
:1076B00050461B1A99400A43511E8A414B460021ED
:1076C0001A439FE6002E30D126003E4367D0DB43AD
:1076D0009A46002B1CD0614EB04260D05346382BE6
:1076E00000DD96E01F2B00DD9FE02026F31A260028
:1076F0009E409C46B34653463E00DE4033005E4605
:107700001E4363469F407B1E9F415346DC403743E8
:10771000BF189742924164185242A418060078E6B6
:1077200027437C1EA741002437E74C4EB04236D099
:1077300080265B4236049A463443CFE71800104354
:1077400000D103E6B81A84466745AD41E01A6D42A0
:10775000401B050200D42CE6D71BBA4292411C1BE9
:107760005242A41AD846F1E51800104300D163E74D
:10777000F808670707438020E4080003044208D0A4
:10778000DD08054205D1D208590711430F002C002E
:10779000D8467B0FE4001C43FF00304ED6E50C00BA
:1077A00017000600D2E5002B38D00B00134300D1A0
:1077B00042E7F808670707438020E4080003044213
:1077C000E7D0CB080342E4D1D208490711430F00A8
:1077D0001C00DEE700270024D5E500216BE700252B
:1077E0000027F3E54E462500203EF5404B462E008F
:1077F000202B2DD04025ED1AAC4027437C1EA741FD
:1078000000243743C9E6802400252403134E0027B3
:10781000DCE527437C1EA741002479E70C00170014
:107820000E4E93E50C00170090E556462300203ECF
:10783000F34099465346202B0ED0402356469B1BBF
:107840009C4027437C1EA7414B4600241F435FE713
:107850000024D2E71700B2E50024F2E7FF0700009A
:10786000FFFF7FFFF0B557464546DE464E46E0B582
:107870004C000E0387B0834692461D008046360BAF
:10788000640DCF0F002C4FD06F4B9C4235D080231E
:10789000420F1B04F600134333439946C300984636
:1078A0006A4B00269C460023644403932B031B0B66
:1078B0009B466B00ED0F50465B0D01955ED0624A12
:1078C000934253D05A46D1008022400F1204024303
:1078D0000A4393465246D1005C4A944600226344D0
:1078E0003800684084460290E41A16430F2E00D9EF
:1078F000B4E0574BB6009B599F460300334399466B
:107900006CD100239846023308260393CEE7CB467A
:107910004146039A0197022A65D1019B4A4C9C4635
:107920000023002298466BE00300334399464ED073
:10793000002E00D1BCE1300001F07EFA03000B3BC9
:107940001C2B00DDACE11D22D31A5A460100DA409F
:1079500008398E401300334399465B468B40984666
:1079600000233C4C0026241A03939FE751465A46B5
:10797000114329D1002293460232B1E7594601430F
:107980001ED05B46002B00D19EE1584601F054FA10
:1079900003000B3B1C2B00DD8FE102005946083A27
:1079A00091408B461D21CB1A5146D9400B005946B8
:1079B0000B4351469B469140264B00221B1A8FE7F2
:1079C000002301229B468BE75146032288E70023D0
:1079D0009846013304260024039367E70323B14646
:1079E00003930C2662E7032A00D15CE2019B012A83
:1079F00000D0E4E113409C46002300240022984676
:107A000000211203130B0A0D12051A432305124C11
:107A100040462240134362465B00D2075B08134393
:107A2000190007B03CBC90469946A246AB46F0BD53
:107A3000002380229C4612039846034CE0E7002373
:107A4000014C00229846DBE7FF07000001FCFFFF26
:107A5000509800000DFCFFFFFFFF0F80D94500D9B3
:107A600039E100D134E1002346464D469A46013CB7
:107A70005B460A0E1B021A430B02170C03931304F6
:107A80001B0C3900280090460193FEF7D3FC02003E
:107A9000019B83465A43280039009146FEF750FD6A
:107AA000350C09040D43A9450DD95B464544013BFE
:107AB000A84500D93AE1A94500D837E102235B4245
:107AC0009C464544E3444B46EB1A390018000493A6
:107AD000FEF7B0FC019B050043433900049899462A
:107AE000FEF72EFD330409041B0C0B43994509D9FD
:107AF00043446A1E984500D91AE1994500D817E118
:107B0000023D43444A469B1A5A4612042A430399AB
:107B10009346100C0A0C914609045A46090C4E462D
:107B20000D001204120C45430591514372437043FA
:107B300052190E0CB218954203D980256D02AC463D
:107B40006044150C09041204090C281852188342C9
:107B500000D2CEE000D1C8E01D1A53469E1AB245AD
:107B600092415242AB1A9A46984500D117E139002A
:107B70001800FEF75FFC019B0500434339005046A7
:107B80000493FEF7DDFC04980B04310C1943884282
:107B900009D941446B1E884500D907E1884200D8C5
:107BA00004E1023D4144049BCB1A180039000493C0
:107BB000FEF740FC019B8246434339000498019341
:107BC000FEF7BEFC01980B043104090C19438842EE
:107BD0000DD953464144013B884500D9E8E088422D
:107BE00000D8E5E002235B429C464144E244019B0D
:107BF0002D04CE1A51462943059D4F462A000B04F9
:107C0000080C1B0C5A4345437B4378435B19170C04
:107C1000FB189D4203D980256D02AC4660441D0CC3
:107C200012041B04120C28189B18864200D293E001
:107C300000D18EE001231943A04BE318002B00DC98
:107C400099E04A0700D09EE05A46D20106D55A462E
:107C50009B4B1A4080239346DB00E318994A9342DA
:107C600068DD0123029A984C1A40002394469846F6
:107C70000022C5E680224B46120313420AD05B461F
:107C8000134206D11A431203120BAC4688468E4C9F
:107C9000B6E64B461A431203120BBC468A4CAFE6BB
:107CA00003005A46283B9A4000239146984657E6DF
:107CB000584601F0C1F8203040E603005246283B08
:107CC0009A400021934677E601F0B6F820305FE64F
:107CD000884500D2C7E64B46DE075D0843465B0891
:107CE0001E434346DB079A46C2E60025924500D371
:107CF00033E7039E5946B446E244B245AD416D4276
:107D00004544EB180139984507D2984200D97FE0E5
:107D100000D1BCE01D1A8B461FE79845FAD1039DA0
:107D20005545F2D943468B461D1A16E79B46CAE6CF
:107D30001500E7E65A46C90852070A435B05904614
:107D40005C0D5A460123029952021940120B8C46CF
:107D500056E6002B00D16FE746444A1EB04529D9AC
:107D60001100864200D065E7039A934200D061E794
:107D700062E7012149420120C21A382A21DD029B13
:107D800003409C4638E60F220A40042A00D15BE7F4
:107D90000A00111D914292415242934454E7474BCD
:107DA000E318002BE5DD01225242F2E71D00FAE65E
:107DB0009A461CE7B04239D86ED011003AE70293D8
:107DC0003AE71F2A3CDC20239B1A0C0058469940B6
:107DD00098404B1E99415B46D440D3402043084312
:107DE0001A00430709D00F230340042B05D00100DC
:107DF000081D88429B415B42D21813023AD50123E9
:107E0000029A01241A400023944698460022F7E57E
:107E1000022149428C46039DE344AC46E244AA4514
:107E2000AD416D424544ED182D1A96E68A1E039920
:107E30004D008D42894149424144761803958FE7B0
:107E40001F204042C31A5846D8400300202A28D099
:107E500040205D46821A954029434A1E91411943AC
:107E6000072300220B4009D00F2300220B400800FB
:107E7000042BBDD1010053075202120BC90819434C
:107E8000012388460299002419408C46B8E55245E2
:107E9000BED88B46002560E6039D9D42C6D31100E7
:107EA00062E70025D8E780225B4612031A43019B54
:107EB0001203120B9C468846034CA1E5FF03000009
:107EC000FFFFFFFEFE070000FF070000F0B54F4672
:107ED0004646D6465C00C0B51F03DB0F9A46174BDB
:107EE0000E034D0084468046360B6D0DC90F91463A
:107EF0003F0B640D01209D4208D09C4201D0A54259
:107F00000BD01CBC90469946A246F0BD6346334355
:107F1000F7D1AC42F5D13A43F3D10120BE42F0D1C2
:107F2000C845EED1514507D0002DEAD163461E4326
:107F30003000461EB041E4E70020E2E7FF07000002
:107F4000F0B54546DE4657464E46E0B51F033D0BAD
:107F50002C4F0E034C00AB465D008446360B640D7F
:107F6000C90F90466D0DDB0FBC422AD0254FBD4294
:107F70002DD0002C0FD13043070081467842784144
:107F8000C0B2002D17D15F463A4314D14B460020B2
:107F9000002B0AD006E0002D02D15846024301D042
:107FA000994218D04842012108433CBC904699466A
:107FB000A246AB46F0BD0028F2D00120013B184399
:107FC000F3E737000743D1D002204042EDE75F4698
:107FD0001743CED0F8E7AC42E4DC03DA481E0121B7
:107FE0000843E2E75E45DDD806D000205E45DCD2DE
:107FF0000123481E1843D8E7C445D3D80020C44500
:10800000F6D3D2E7FF070000F0B54E464546DE4600
:1080100057465C00E0B51F03DB0F99462A4B0E0361
:108020004D00C90F8446360B6D0D8B4690463F0BB5
:10803000640D9D4220D0244B9C4222D0002D12D1B1
:10804000304343424341DBB2002C1FD0002B0CD005
:108050004B460120013B034318003CBC9046994627
:10806000A246AB46F0BD002C16D0CB4517D05B46E0
:10807000594201230B43EFE7310002230143EBD1C7
:10808000D9E7390002231143E6D1D7E73A43DDD1DE
:1080900000230028E0D0EAE73A43E6D1E7E7A5422B
:1080A000E5DC05DBBE42E2D807D00023BE42D3D2D6
:1080B0005946012301390B43CEE7C445D7D80023E5
:1080C000C445F5D3C8E7C046FF070000F0B55746E2
:1080D0004546DE464E46E0B50C0398464E00230B5F
:1080E00087B0070092469B46760DCD0F002E6BD0D1
:1080F0006D4B9E4235D080245B46420F2404DB004A
:1081000014431C43C3009946684BA3469C46002376
:1081100000276644029343461C035A00DB0F504677
:10812000240B520D984600D176E05F4B9A426DD0F9
:108130008023410F1B040B435C49E4008C461C4325
:10814000C300002062444146B6186940721C019188
:10815000944607430F2F00D9B0E0554ABF00D259CB
:1081600097465B460343994600D087E000239B4631
:10817000023308270293CEE742460192022867D0D5
:10818000032800D10EE2012800D062E10023002480
:108190000022994601990140CDB2002112030B0D36
:1081A000120B1B051343434A240513401C43640070
:1081B000ED0764082C434846210007B03CBC9046BC
:1081C0009946A246AB46F0BD034399464FD05B4665
:1081D000002B00D189E1584600F02EFE03000B3B36
:1081E0001C2B00DD7AE11D22D31A3A0001005C4607
:1081F000DA4008398C4013008F4023439B46B94630
:1082000000232D4E0027361A029384E7534623435A
:108210002AD10024022096E75346234320D0002C85
:1082200000D157E1200000F007FE03000B3B1C2BA0
:1082300000DD49E11D21CB1A51460200D9405346C9
:10824000083A944093400C431B4A121A00207AE7E4
:108250000125019B144C1D400023002299469CE7F8
:108260000024002201206EE7534603206BE7002321
:108270009B4601330427002602934CE703238146E3
:108280000C27029347E7802200230025120399461A
:10829000054C82E75C464B4602986FE75C464B46CE
:1082A000019502986AE7C046FF07000001FCFFFF46
:1082B00090980000FFFF0F800DFCFFFF4A464946E3
:1082C000170C1A0C1B041B0C08041900000C41436A
:1082D0001500884619007D43794303958946290096
:1082E000150045434D44029545462D0CAA46029D76
:1082F0005544A94506D98A46802149028946CA447F
:1083000051460391290C0491414609042D04090C9E
:1083100088462900250C24044144240C05912100A1
:1083200041438846210079438A4668434146504488
:108330008146080C48446F43824503D98021490295
:1083400089464F44010C894639004944029141460F
:108350000F0404993F0C88460004C019804441462C
:10836000049159460F0C0904090C884659438A4662
:1083700039005143894641464A435146090C8B46D0
:108380007B43D2185A44934203D980235B029B4615
:10839000D94451460904090C8A46414661437C434D
:1083A000130C12044B445244A1468A463C004146F9
:1083B0006C434D4351464D440F0C7D19A94503D9DB
:1083C0008021490288464444049F0399B8464144A9
:1083D0008B468345804141428846514608042F041C
:1083E000000C3F1858460299101889469042924155
:1083F0004F44BA46524299469346C244D144CB4474
:108400008F42BF41C245894199459B419345924165
:108410007F4249422D0C52420F435B4213437F1966
:10842000FF185B463C19DB0D059A64021C434302AE
:1084300013435D1EAB415A46C00D03435202134322
:10844000E20156D501205A0803401343E2071343C3
:1084500064085A48604400284DDD5A0709D00F22AD
:108460001A40042A05D01A1D9A429B415B42E41827
:108470001300E20104D58020514AC000144060443A
:10848000504A904200DDE3E60125DB0862071A430B
:108490006402019B9146220B4405640D1D407CE65D
:1084A000802259461203114208D0144206D12243B9
:1084B0001203120B45469946434C6EE65B461A433F
:1084C0001203120B404C68E603005446283B9C40C4
:1084D0000023B9E600F0B0FC2030A6E60300283BFC
:1084E0009F400023BB4699468AE600F0A5FC203059
:1084F00074E6B446ADE701252A1A382A06DD019B49
:1085000000241D4000230022994646E61F2A21DC54
:1085100020252000AD1A1E00AB40A840D6405D1EAD
:10852000AB4130431843D440430709D00F230340E5
:10853000042B05D00300181D98429B415B42E418B0
:10854000230221D50125019B01241D400023002287
:10855000994622E61F2521006D42281AC1400800D5
:10856000202A1DD05F35AA1A944023435C1EA341E4
:10857000072503431D400022002D09D00F220024AF
:108580001A401800042AD6D1030065076402220BA2
:10859000DB082B4301259946019B00241D40FCE587
:1085A0000024E2E7802201251203224301991203ED
:1085B000120B0D409946044CEFE5C046FF03000046
:1085C000FFFFFFFEFE070000FF070000F0B5464674
:1085D000D6464F460C03C0B5CD0F4E00610A440F7E
:1085E0000C43C1005800400D84468A460F00190311
:1085F000500F490A0143C648760DA846DB0FD2004A
:10860000844500D1D8E001204340AB4200D1A6E030
:108610006046351A002D00DC05E1002810D10B0062
:10862000134300D1D7E06B1E002B00D04BE1534623
:108630009F1ABA458041641A4042241A01261EE05E
:10864000B34B9E4248D080231B041943382D00DDD4
:1086500019E11F2D00DD4CE120230F005B1B1000F2
:108660009A409F40E840531E9A41E9400743174310
:108670005346DF1B611ABA45A44164420C1B230216
:1086800000D4C5E06402650A002D00D1F6E02800A0
:1086900000F0D2FB0300083B1F2B00DDE9E02022A5
:1086A0003C00D21A9D40D4409F4025439E4200DDAD
:1086B000DBE09E1B731C1F2B00DD0AE1202238002B
:1086C000D21A290097402C009140D8407A1E974139
:1086D000DC40002601430F437B0709D00F233B40BA
:1086E000042B05D03B1DBB42BF417F42E4191F0054
:1086F000230225D5864B01369E4200D1AFE0854B43
:1087000001251C4043466207FF08640276051743B3
:10871000240B760D1D4000212403230B0C0D7E4AF3
:1087200024051C431440330523435B00ED075B081D
:108730002B43380019001CBC90469946A246F0BD58
:10874000012543466207FF081743E4081D40704BAC
:108750009E4236D024037605240B760DDBE7634674
:10876000F31A002B00DC94E06046002835D06848FE
:108770008642B1D080273F043943382B00DCFDE02E
:108780000A43170000217A1E9741574457458041FC
:10879000091944420C1923023AD55D4B01369E4219
:1087A00000D14BE101225B4B1C407B0817401F436B
:1087B000E207174364088FE70800104300D024E75E
:1087C00021E723003B4300D1B9E180221203144387
:1087D0002403240B9FE72E007EE70800104300D1FE
:1087E000CAE0581E8446002800D0E7E052445245B3
:1087F000804164184042241817000126230207D53F
:108800000226CFE764462C4300D1B3E12C00674633
:108810007B0700D062E76307FF081F43012543463B
:10882000E4081D4093E7002D78D1751C6D056D0D92
:10883000012D00DCF2E05046801A8245BF41651AE6
:108840007F42ED1B8446280200D48CE05046171A64
:10885000BA4292410C1B5542651B984614E701250C
:10886000434600241D40002755E72A4CF61A2C40A9
:1088700032E73D0028388540002717E7380000F030
:10888000DBFA203006E70A43170000217A1E9741E1
:10889000EEE6002B00D0E5E0731C9C465B055B0D0B
:1088A000012B00DC9FE01A4B9C4500D1C5E05244EF
:1088B00052458041641840422418E7075208174384
:1088C0006408664608E71248854200D185E01D002D
:1088D000BCE629001F3EF140202B00D17FE0402262
:1088E000D31A9D402F437D1EAF4100240F43002625
:1088F0008EE72B000F00203BDF40202D71D040235E
:108900005D1BA9400A43511E8A4100211743AFE66F
:10891000FF070000FFFF7FFFFFFF0F80002E3ED00C
:10892000B34EB44545D0802636046D423443382DCD
:1089300000DDA8E01F2D00DD1FE1202627005046A6
:10894000761BB740E84007435046B040461EB04152
:10895000EC403843171ABA4292410C1B5242A41AF7
:10896000664698468BE6644667462C4300D08BE605
:10897000002500260027EAE61E00ADE61F2B60DC7E
:108980002027F81A0F00844687401000D84007437C
:1089900060468240501E8241D9401743F5E62600CA
:1089A0005046064305D0ED43002DD3D0904EB4453C
:1089B000BDD10C001700664698468DE68C48834270
:1089C0000BD06346D9E6002D00D096E00800104396
:1089D00000D1E2E00C0017009846854E7CE60025A9
:1089E00080E700218EE7230050460343002E00D08D
:1089F000A8E0002B00D1DEE00B00134300D16BE6B2
:108A00005244524580416418404224181700230202
:108A100000D4FDE6774B66461C405DE625005046D7
:108A20000543002ECFD1002D4FD10C00144300D1AF
:108A3000A0E00C00170098464EE66646002400278A
:108A400085E61F000800203FF8400700202B00D1DA
:108A50008EE04020C31A99400A43511E8A410021EA
:108A6000174392E6002E14D126005046064362D0EA
:108A7000DB43002B5CD18718974292416418524225
:108A8000A418664687E650462043441EA0410024B1
:108A900060E7574EB4454ED0802636045B423443DF
:108AA000382B00DD7FE01F2B00DD8BE02026270028
:108AB0005046F61AB740D84007435046B040461ECD
:108AC000B0410743DC40BF18D6E70D00154300D185
:108AD00002E65046801A8245BF41651A7F42ED1B6F
:108AE0008446280200D48DE65046171ABA429241B5
:108AF0000C1B5242A41A9846EEE50D00154300D116
:108B00006BE750466707C00807438020E40800036E
:108B1000044207D0CD08054204D12C009846D7085E
:108B200049070F437B0FE4001C43FF00304ED3E5A1
:108B30002F4EB445B4D10C0017006646CCE5002793
:108B40000024E8E5002B39D00B00134300D144E7A3
:108B5000C008670707438020E40800030442E1D00F
:108B6000CB080342DED1D70849070F431C00D9E7E1
:108B7000002171E700250027E9E52E002700203EAF
:108B8000F740202D2FD04026751BAC405046204387
:108B9000441EA04100243843DCE680240025240341
:108BA000134E0027D3E5504620430700781E874127
:108BB0000024BF1860E70C0017008DE50C001700BB
:108BC0000B4E89E51E002700203EF740202B0CD0DD
:108BD0004026F31A9C4050462043441EA0410743C0
:108BE0000024BF1848E70024D0E70024F3E7C0467C
:108BF000FF070000FFFF7FFF70B50E4E0D031C0343
:108C000049005B002D0B490D240B5B0DB14204D0D4
:108C1000084900208B4208D070BD05430120002D7B
:108C2000FAD1044900208B42F6D114432000441E9F
:108C3000A041F1E7FF07000030B5134D0A034B00D8
:108C4000120B5B0DC90F0024AB4210DD0F4CA34289
:108C50000FDC80240E4D64032243ED1A1F2D0BDD23
:108C60000C48C31ADA405442002900D114002000F5
:108C700030BD094BCC18FAE7084CE840A4466344E1
:108C80009A400243EFE7C046FE0300001D040000C7
:108C90003304000013040000FFFFFF7FEDFBFFFF24
:108CA00070B5002830D0C317C4185C40C50F200031
:108CB00000F0C2F8174B184A1B1AD21A1F2A18DDE7
:108CC000164AD21A9440002224035B05240B5B0D44
:108CD0000021100024030A0D240B12052243104C1E
:108CE0001B05224013435B00ED075B082B43190073
:108CF00070BD210091400A000B21081AC4405B0599
:108D00002403240B5B0DE3E700250023002400224D
:108D1000DEE7C0461E040000330400001304000018
:108D2000FFFF0F8010B5041E28D000F085F8154B0A
:108D3000154A1B1AD21A1F2A15DD144AD21A94405A
:108D4000002224035B05240B5B0D0021100024038B
:108D50000A0D240B120522430D4C1B052240134320
:108D60005B00590810BD210091400A000B21081A30
:108D7000C4405B052403240B5B0DE6E700230024BD
:108D80000022E2E71E040000330400001304000088
:108D9000FFFF0F804100090E4B1C70B5DBB246028D
:108DA000750AC40F012B14DDE0239B006D07360B01
:108DB000CB1800210A0D280012051C4D32435B051B
:108DC0002A405B0813435B00E4075B082343190058
:108DD00070BD002914D1002D1ED0280000F02CF801
:108DE0000A281CDC0B232A001B1ADA400300153367
:108DF0009D400F4B12031B1A5B05160B5B0DD8E74A
:108E0000002D06D0320B802636036D071643094B22
:108E1000CFE7084B0026CCE700230026C9E7030074
:108E20002A000B3B9A400025E3E7C046FFFF0F8076
:108E300089030000FF0700001C2101231B04984246
:108E400001D3000C10391B0A984201D3000A0839DB
:108E50001B09984201D30009043902A2105C401892
:108E60007047C04604030202010101010000000036
:108E70000000000010B5002903D1FFF7DDFF20300E
:108E800002E0081CFFF7D8FF10BDC0460D2300000C
:108E90000D2040005941524D20496E697420446FA5
:108EA0006E652E2E2E0D00005941524D20506F77C9
:108EB00065724F6E20446F6E652E2E2E0D000000E1
:108EC00025635B34376D000025635B33316D000033
:108ED0004572726F722061742025732C2045727266
:108EE0006F72436F64653A2025640D0A000000002C
:108EF00025635B306D000000446F6E652025732094
:108F00005B3078255820307825585D0D0A00000028
:108F10005941524D5F4C6962733A2044617461203B
:108F20005265636569766564205B33325D0D0000D0
:108F30002030782530582C20000000005941524D37
:108F40005F53657449646C654D6F64650000000093
:108F50005265672E204745544556454E5442595454
:108F600045533A2000000000307825582C2000009E
:108F70005941524D5F53657453797374656D4D6FEC
:108F800064652054584D6F64650000005941524D8E
:108F90005F57726974655478507265616D626C6573
:108FA000000000005941524D5F5772697465547852
:108FB0004669666F0000000054584C6F6F70205374
:108FC0007461727465640D0054584C6F6F70204565
:108FD0006E646564206174206379636C65203A2057
:108FE0002564205B2564206D735D0D0A0000000080
:108FF000545820456E646564206F6E2073657276E8
:109000006963653A202564206368616E6E656C3A19
:109010002025640D0A0000009C0E0000CC1000000A
:10902000CC100000CC100000CC100000CC100000D0
:10903000CC100000CC100000CC100000CC100000C0
:10904000CC100000CC100000CC100000CC100000B0
:10905000CC100000CC100000840E0000CC100000EA
:10906000CC100000CC100000CC100000CC10000090
:10907000CC100000CC100000CC100000CC10000080
:10908000CC100000CC100000CC100000CC10000070
:10909000CC100000CC100000940E0000CC1000009A
:1090A000CC100000CC100000CC100000CC10000050
:1090B000CC100000CC100000CC100000CC10000040
:1090C000CC100000CC100000CC100000CC10000030
:1090D000CC100000CC1000008C0E0000A40E00008C
:1090E0006C0E00007C0E0000740E000002000000F8
:1090F00003000000FFFF0000FFFF0000040000006D
:10910000050000000600000007000000FFFF00004F
:10911000FFFF0000FFFF0000FFFF0000FFFF000057
:10912000FFFF0000FFFF0000FFFF0000080000003D
:10913000090000000A0000000B000000FFFF000013
:10914000FFFF0000FFFF0000FFFF00003078253028
:10915000327820004552524F523A2041636B206EC4
:109160006F74207265636569766564202120212013
:1091700021200D000D0A0D0A2D2D2D2D20525820D5
:1091800066726F6D205941524D20434D33202D2D75
:109190002D2D2D2D2D2D2D2D2D2D2D2D2D2D2D2DFF
:1091A0000D000000526563656976656420256420C2
:1091B0006279746573206F6E20736572766963657A
:1091C000202564206368616E6E656C2025640D0A3D
:1091D000000000004E6F64653A20446174612052C3
:1091E00065636569766564205B25645D0D0A000032
:1091F0003078253032582000434D3349443A2030EE
:10920000782530345825303458253034580D0A002C
:109210004E756D204D65737361676520526563659A
:10922000697665643D2025640D0A00005253534958
:109230002052656365697665642066726F6D2043B0
:109240004D333A20252E32662064426D0D0A00000F
:10925000525353493A20252E32662064426D0D0A3E
:1092600000000000566F6C746167652F436F6D6D71
:10927000616E64203D2025642028307825303478C4
:10928000290D0A0052784572726F723A2025640DDA
:109290000A0000000D0A0D000D0A0D0A2D2D2D2DBE
:1092A00020545820746F205941524D20434D332093
:1092B0002D2D2D2D2D2D2D2D2D2D2D2D2D2D2D2DDE
:1092C0002D2D0D004461746120746F2053656E6410
:1092D000205B25645D0D0A004E756D204D6573732E
:1092E000616765203D2025640D0A000030393A355C
:1092F000313A3233000000004A616E2020332032C0
:10930000303138002020202020202020202020590B
:1093100041524D204861727665737431203132209C
:109320003230313720636F6D6D6F6E204C69627320
:109330002025732025730D0A0000000053656E730D
:109340006F722044617461205061636B6574204CBE
:10935000656E677468203D2025640D0A00000000DA
:1093600053657269616C4E756D6265723A20305852
:109370002025307820253078202530782025307839
:109380000D0A00005941524D5F496E69740D00008D
:10939000456E74657220536C656570203220746967
:1093A0006D656F7574203D202564206D730D0A0076
:1093B0004E65772073656E6420706572696F6420F6
:1093C0003D202564206D730D0A000000252E3266B5
:1093D0000000000054696D6572204576656E742149
:1093E000202061646373616D706C65203D2030786E
:1093F0002530347820282564292056203D20252E2C
:1094000032665620627566766F6C74616765203DC2
:1094100020257320525353495F72656365697665F1
:1094200064203D20252E3031662064426D0D0A00F7
:10943000456E64206F662054780D0A57616974691F
:109440006E672041636B0D00000000420004004283
:1094500000080042000C00420010004200040043DB
:109460003E2F00003A2F00003A2F0000A02F0000EE
:10947000A02F0000542F0000442F00005A2F00009E
:109480008E2F0000EC2F0000CC2F0000CC2F00000E
:1094900066300000DE2F0000FA2F0000D02F000001
:1094A000083000004A300000A4300000E630000020
:1094B000E6300000E630000096300000B2300000D8
:1094C00088300000C0300000D6300000600000206E
:1094D000494E4600696E66004E414E006E616E0058
:1094E0003000303132333435363738394142434435
:1094F00045460030313233343536373839616263AE
:1095000064656600496E66696E697479004E614EE5
:10951000000000000000000000000000000000004B
:10952000000000000000000000000000000000003B
:10953000000000000000000000000000000000002B
:10954000000000000000000000000000000000001B
:10955000000000000000000000000000000000000B
:1095600000000000000000000000000000000000FB
:1095700000000000000000000080E03779C3414394
:10958000176E05B5B5B89346F5F93FE9034F384D69
:10959000321D30F94877825A3CBF737FDD4F157515
:1095A000000000000000F03F000000000000244028
:1095B00000000000000059400000000000408F4003
:1095C000000000000088C34000000000006AF8406E
:1095D0000000000080842E4100000000D012634192
:1095E0000000000084D797410000000065CDCD4108
:1095F000000000205FA00242000000E876483742E9
:10960000000000A2941A6D42000040E59C30A24286
:109610000000901EC4BCD64200003426F56B0C43FB
:109620000080E03779C3414300A0D88557347643A2
:1096300000C84E676DC1AB43003D9160E458E14303
:10964000408CB5781DAF154450EFE2D6E41A4B4478
:1096500092D54D06CFF08044F64AE1C7022DB544BD
:10966000B49DD9794378EA44050000001900000050
:109670007D000000232D302B2000686C4C006566B7
:1096800067454647004300504F534958002E00009D
:1096900020202020202020202028282828282020A2
:1096A00020202020202020202020202020202020BA
:1096B0008810101010101010101010101010101032
:1096C0000404040404040404040410101010101012
:1096D00010414141414141010101010101010101EB
:1096E000010101010101010101010110101010101F
:1096F00010424242424242020202020202020202BC
:1097000002020202020202020202021010101020E3
:109710000000000000000000000000000000000049
:109720000000000000000000000000000000000039
:109730000000000000000000000000000000000029
:109740000000000000000000000000000000000019
:109750000000000000000000000000000000000009
:1097600000000000000000000000000000000000F9
:1097700000000000000000000000000000000000E9
:1097800000000000000000000000000000000000D9
:109790003C6B00000C6B00001E6B0000606A000058
:1097A0001E6B0000026B00001E6B0000606A000070
:1097B0000C6B00000C6B0000026B0000606A000084
:1097C000686A0000686A0000686A0000246B000094
:1097D0000C6B00000C6B0000E06A0000C46B000022
:1097E000E06A0000026B0000E06A0000C46B000049
:1097F0000C6B00000C6B0000026B0000C46B0000DF
:10980000686A0000686A0000686A0000CE6B0000A9
:109810006C6D0000BC6C0000BC6C0000BA6C0000F9
:109820005E6D00005E6D0000546D0000BA6C0000BB
:109830005E6D0000546D00005E6D0000BA6C0000AB
:10984000646D0000646D0000646D0000F46D000044
:109850005C7A00003E7A0000F8790000167900007A
:10986000F8790000307A0000F879000016790000DD
:109870003E7A00003E7A0000307A0000167900003F
:109880000E7900000E7900000E790000747C000053
:10989000BC8200007C8100007C8100007881000097
:1098A000948200009482000086820000788100008B
:1098B000948200008682000094820000788100007B
:1098C0009C8200009C8200009C820000A08400001A
:1098D000F8B5C046F8BC08BC9E467047DD000000E5
:1098E000F8B5C046F8BC08BC9E467047B5000000FD
:0898F00040CFFF7F01000000E2
:1098F800BFF35F8F01380028FAD1704700000000DD
:109908000078786E7837006E6E37320000000000FD
:1099180000004155000032370046460004708E0AA8
:109928005555105556000000405060415161425253
:1099380062435363445464000CA0800040A080003C
:10994800E803000088130000010000006000002008
:1099580000000000349500005495000014950000A4
:1099680000000000000000000000000000000000EF
:1099780000000000000000000000000000000000DF
:1099880000000000000000000000000000000000CF
:1099980000000000000000000000000000000000BF
:1099A80000000000000000000000000000000000AF
:1099B800430000000000000000000000000000005C
:1099C800000000000000000000000000000000008F
:1099D800430000000000000000000000000000003C
:1099E800000000000000000000000000000000006F
:1099F800430000000000000000000000000000001C
:109A0800000000000000000000000000000000004E
:109A180043000000000000000000000000000000FB
:109A2800000000000000000000000000000000002E
:109A380043000000000000000000000000000000DB
:109A4800000000000000000000000000000000000E
:109A580043000000000000000000000000000000BB
:109A680000000000000000000000000000000000EE
:109A7800430000000000000000000000000000009B
:109A880000000000000000000000000000000000CE
:109A9800F96300003D630000000000008F9600009D
:109AA8008D9600007996000079960000799600005E
:109AB8007996000079960000799600007996000062
:109AC8007996000079960000FFFFFFFFFFFFFFFF78
:109AD800FFFFFFFFFFFF000001004153434949001A
:109AE800000000000000000000000000000000006E
:109AF80000000000000000000000415343494900F5
:109B0800000000000000000000000000000000004D
:0C9B180000000000000000000000000041
:0400000300003519AB
:00000001FF
